Archive member included because of file (symbol)

c:/program files/microchip/mplab c30/bin/../lib\libpic30-coff.a(crt1.o)
                              (_resetALT)
c:/program files/microchip/mplab c30/bin/../lib\libpic30-coff.a(crt0.o)
                              (_resetPRI)
c:/program files/microchip/mplab c30/bin/../lib\libc-coff.a(printf.io)
                              loopback.o (_iprintf)
c:/program files/microchip/mplab c30/bin/../lib\libc-coff.a(islower.os)
                              ping_app.o (islower)
c:/program files/microchip/mplab c30/bin/../lib\libc-coff.a(toupper.os)
                              ping_app.o (toupper)
c:/program files/microchip/mplab c30/bin/../lib\libc-coff.a(memset.o)
                              ping_app.o (memset)
c:/program files/microchip/mplab c30/bin/../lib\libc-coff.a(puts.o)
                              ping_app.o (puts)
c:/program files/microchip/mplab c30/bin/../lib\libc-coff.a(strtok.o)
                              ping_app.o (strtok)
c:/program files/microchip/mplab c30/bin/../lib\libc-coff.a(strcmp.o)
                              ping_app.o (strcmp)
c:/program files/microchip/mplab c30/bin/../lib\libc-coff.a(strchr.o)
                              ping_app.o (strchr)
c:/program files/microchip/mplab c30/bin/../lib\libc-coff.a(strlen.o)
                              ping_app.o (strlen)
c:/program files/microchip/mplab c30/bin/../lib\libc-coff.a(strcpy.o)
                              ping_app.o (strcpy)
c:/program files/microchip/mplab c30/bin/../lib\libc-coff.a(strstr.o)
                              webserver.o (strstr)
c:/program files/microchip/mplab c30/bin/../lib\libc-coff.a(memcpy.o)
                              webserver.o (memcpy)
c:/program files/microchip/mplab c30/bin/../lib\libc-coff.a(sprintf.io)
                              webserver.o (_isprintf)
c:/program files/microchip/mplab c30/bin/../lib\libc-coff.a(memcmp.o)
                              config.o (memcmp)
c:/program files/microchip/mplab c30/bin/../lib\libc-coff.a(strcat.o)
                              dns.o (strcat)
c:/program files/microchip/mplab c30/bin/../lib\libc-coff.a(fwrite.o)
                              c:/program files/microchip/mplab c30/bin/../lib\libc-coff.a(printf.io) (fwrite)
c:/program files/microchip/mplab c30/bin/../lib\libc-coff.a(xfiles.o)
                              c:/program files/microchip/mplab c30/bin/../lib\libc-coff.a(printf.io) (_Stdout)
c:/program files/microchip/mplab c30/bin/../lib\libc-coff.a(xprintf.io)
                              c:/program files/microchip/mplab c30/bin/../lib\libc-coff.a(printf.io) (__iPrintf)
c:/program files/microchip/mplab c30/bin/../lib\libc-coff.a(fputs.o)
                              c:/program files/microchip/mplab c30/bin/../lib\libc-coff.a(puts.o) (fputs)
c:/program files/microchip/mplab c30/bin/../lib\libc-coff.a(fputc.o)
                              c:/program files/microchip/mplab c30/bin/../lib\libc-coff.a(puts.o) (fputc)
c:/program files/microchip/mplab c30/bin/../lib\libc-coff.a(strspn.o)
                              c:/program files/microchip/mplab c30/bin/../lib\libc-coff.a(strtok.o) (strspn)
c:/program files/microchip/mplab c30/bin/../lib\libc-coff.a(strcspn.o)
                              c:/program files/microchip/mplab c30/bin/../lib\libc-coff.a(strtok.o) (strcspn)
c:/program files/microchip/mplab c30/bin/../lib\libc-coff.a(xfwprep.o)
                              c:/program files/microchip/mplab c30/bin/../lib\libc-coff.a(fwrite.o) (_Fwprep)
c:/program files/microchip/mplab c30/bin/../lib\libc-coff.a(memchr.o)
                              c:/program files/microchip/mplab c30/bin/../lib\libc-coff.a(fwrite.o) (memchr)
c:/program files/microchip/mplab c30/bin/../lib\libc-coff.a(fflush.o)
                              c:/program files/microchip/mplab c30/bin/../lib\libc-coff.a(fwrite.o) (_DNKfflush)
c:/program files/microchip/mplab c30/bin/../lib\libc-coff.a(xvacopy.o)
                              c:/program files/microchip/mplab c30/bin/../lib\libc-coff.a(xprintf.io) (_Vacopy)
c:/program files/microchip/mplab c30/bin/../lib\libc-coff.a(xputfld.io)
                              c:/program files/microchip/mplab c30/bin/../lib\libc-coff.a(xprintf.io) (__iPutfld)
c:/program files/microchip/mplab c30/bin/../lib\libc-coff.a(xputtxt.o)
                              c:/program files/microchip/mplab c30/bin/../lib\libc-coff.a(xprintf.io) (_Puttxt)
c:/program files/microchip/mplab c30/bin/../lib\libc-coff.a(strrchr.o)
                              c:/program files/microchip/mplab c30/bin/../lib\libc-coff.a(fputs.o) (strrchr)
c:/program files/microchip/mplab c30/bin/../lib\libc-coff.a(malloc.o)
                              c:/program files/microchip/mplab c30/bin/../lib\libc-coff.a(xfwprep.o) (malloc)
c:/program files/microchip/mplab c30/bin/../lib\libc-coff.a(fclose.o)
                              c:/program files/microchip/mplab c30/bin/../lib\libc-coff.a(xfwprep.o) (_Closreg)
c:/program files/microchip/mplab c30/bin/../lib\libc-coff.a(xlitob.o)
                              c:/program files/microchip/mplab c30/bin/../lib\libc-coff.a(xputfld.io) (_Litob)
c:/program files/microchip/mplab c30/bin/../lib\libc-coff.a(xgetmem.o)
                              c:/program files/microchip/mplab c30/bin/../lib\libc-coff.a(malloc.o) (_Getmem)
c:/program files/microchip/mplab c30/bin/../lib\libc-coff.a(free.o)
                              c:/program files/microchip/mplab c30/bin/../lib\libc-coff.a(malloc.o) (free)
c:/program files/microchip/mplab c30/bin/../lib\libc-coff.a(xatexit.o)
                              c:/program files/microchip/mplab c30/bin/../lib\libc-coff.a(fclose.o) (_Atexit)
c:/program files/microchip/mplab c30/bin/../lib\libpic30-coff.a(remove.o)
                              c:/program files/microchip/mplab c30/bin/../lib\libc-coff.a(fclose.o) (remove)
c:/program files/microchip/mplab c30/bin/../lib\libpic30-coff.a(sbrk.o)
                              c:/program files/microchip/mplab c30/bin/../lib\libc-coff.a(xgetmem.o) (sbrk)
c:/program files/microchip/mplab c30/bin/../lib\libpic30-coff.a(brk.o)
                              c:/program files/microchip/mplab c30/bin/../lib\libpic30-coff.a(sbrk.o) (brk)
c:/program files/microchip/mplab c30/bin/../lib\libm-coff.a(divmoddi3.o)
                              c:/program files/microchip/mplab c30/bin/../lib\libc-coff.a(xlitob.o) (__udivdi3)
c:/program files/microchip/mplab c30/bin/../lib\libm-coff.a(muldi3.o)
                              c:/program files/microchip/mplab c30/bin/../lib\libc-coff.a(xlitob.o) (__muldi3)
c:/program files/microchip/mplab c30/bin/../lib\libm-coff.a(umuldi3.o)
                              c:/program files/microchip/mplab c30/bin/../lib\libm-coff.a(muldi3.o) (__umuldi3)


Program Memory Usage

section                    address   length (PC units)   length (bytes) (dec)
-------                    -------   -----------------   --------------------
.reset                           0                 0x4             0x6  (6)
.ivt                           0x4                0xfc           0x17a  (378)
.aivt                        0x104                0xfc           0x17a  (378)
.text                        0x200              0x8536          0xc7d1  (51153)
.const                      0x8736              0x4886          0x6cc9  (27849)
.prog                       0xcfbc              0x281e          0x3c2d  (15405)
.dinit                      0xf7da               0xc64          0x1296  (4758)
.isr                       0x1043e                 0x2             0x3  (3)

                     Total program memory used (bytes):        0x1865a  (99930) 75%


Data Memory Usage

section                    address      alignment gaps    total length  (dec)
-------                    -------      --------------    -------------------
.ndata                       0x800                   0          0x1000  (4096)
.ndata                      0x1800                   0            0x88  (136)
.nbss                       0x1888                   0            0x46  (70)
.ndata                      0x18ce                   0            0x40  (64)
.ndata                      0x190e                   0            0x3a  (58)
.nbss                       0x1948                   0            0x34  (52)
.ndata                      0x197c                   0            0x32  (50)
.nbss                       0x19ae                   0            0x2a  (42)
.nbss                       0x19d8                   0            0x28  (40)
.nbss                       0x1a00                   0            0x22  (34)
.ndata                      0x1a22                   0            0x22  (34)
.nbss                       0x1a44                   0            0x20  (32)
.ndata                      0x1a64                   0            0x12  (18)
.nbss                       0x1a76                   0             0xa  (10)
.nbss                       0x1a80                   0             0x8  (8)
.ndata                      0x1a88                   0             0x6  (6)
.nbss                       0x1a8e                   0             0x6  (6)
.ndata                      0x1a94                   0             0x6  (6)
.nbss                       0x1a9a                   0             0x4  (4)
.ndata                      0x1a9e                   0             0x4  (4)
.nbss                       0x1aa2                   0             0x2  (2)
.ndata                      0x1aa4                   0             0x2  (2)
.ndata                      0x1aa6                   0             0x2  (2)
.nbss                       0x1aa8                   0             0x2  (2)
.nbss                       0x1aaa                   0             0x2  (2)
.nbss                       0x1aac                   0             0x2  (2)
.dconst                     0x1aae                   0             0x8  (8)
.dconst                     0x1ab6                   0             0x2  (2)

                        Total data memory used (bytes):         0x12b8  (4792) 58%


Dynamic Memory Usage

region                     address                      maximum length  (dec)
------                     -------                      ---------------------
heap                        0x1ab8                               0x200  (512)
stack                       0x1cb8                               0xb48  (2888)

                        Maximum dynamic memory (bytes):          0xd48  (3400)


External Symbols in Data Memory (by address):

                    0x0800                  _data_buf1
                    0x1000                  _data_buf2
                    0x1800                  __Files
                    0x1810                  __Stderr
                    0x1838                  __Stdout
                    0x1860                  __Stdin
                    0x1888                  _SysInfo
                    0x1892                  _NetConf
                    0x18ac                  _ChConf
                    0x1946                  _romfl_list
                    0x197c                  _GET_DNS_IP
                    0x1980                  _HOST_NAME
                    0x199e                  _GET_SIP
                    0x19a2                  _DHCP_SIP
                    0x19a6                  _DHCP_REAL_SIP
                    0x19aa                  _dhcp_ip_update
                    0x19ac                  _dhcp_ip_conflict
                    0x19ae                  _SRC_MAC_ADDR
                    0x19b4                  _GET_SN_MASK
                    0x19b8                  _GET_GW_IP
                    0x19bc                  _OLD_SIP
                    0x19c0                  _dhcp_state
                    0x19c1                  _retry_count
                    0x19c2                  _DHCP_timeout
                    0x19c4                  _lease_time
                    0x19c8                  _dhcp_time
                    0x19cc                  _next_dhcp_time
                    0x19d0                  _DHCP_XID
                    0x19d4                  _DHCPC_SOCK
                    0x19d6                  _pRIPMSG
                    0x19d8                  _sio_rxd
                    0x19f8                  _sio_head
                    0x19fa                  _sio_tail
                    0x19fc                  _uart_handler
                    0x1a00                  _evb_lcd_text
                    0x1a76                  _dns_buf
                    0x1a78                  _get_domain_name
                    0x1a7a                  _get_domain_ip
                    0x1a7e                  _query_data
                    0x1a80                  _ChannelHandler
                    0x1a88                  _sock_flag
                    0x1a89                  _bchannel_start
                    0x1a8e                  _sys_tick_5ms
                    0x1a90                  _sys_tick_1s
                    0x1a92                  _TIMER_IRQS
                    0x1a94                  __Size_block
                    0x1a96                  __Aldata
                    0x1a9a                  _http_response
                    0x1a9c                  _http_request
                    0x1aa4                  _dns_id
                    0x1aac                  ___curbrk

External Symbols in Data Memory (by name):

                    0x18ac                  _ChConf
                    0x1a80                  _ChannelHandler
                    0x19d4                  _DHCPC_SOCK
                    0x19a6                  _DHCP_REAL_SIP
                    0x19a2                  _DHCP_SIP
                    0x19d0                  _DHCP_XID
                    0x19c2                  _DHCP_timeout
                    0x197c                  _GET_DNS_IP
                    0x19b8                  _GET_GW_IP
                    0x199e                  _GET_SIP
                    0x19b4                  _GET_SN_MASK
                    0x1980                  _HOST_NAME
                    0x1892                  _NetConf
                    0x19bc                  _OLD_SIP
                    0x19ae                  _SRC_MAC_ADDR
                    0x1888                  _SysInfo
                    0x1a92                  _TIMER_IRQS
                    0x1a96                  __Aldata
                    0x1800                  __Files
                    0x1a94                  __Size_block
                    0x1810                  __Stderr
                    0x1860                  __Stdin
                    0x1838                  __Stdout
                    0x1aac                  ___curbrk
                    0x1a89                  _bchannel_start
                    0x0800                  _data_buf1
                    0x1000                  _data_buf2
                    0x19ac                  _dhcp_ip_conflict
                    0x19aa                  _dhcp_ip_update
                    0x19c0                  _dhcp_state
                    0x19c8                  _dhcp_time
                    0x1a76                  _dns_buf
                    0x1aa4                  _dns_id
                    0x1a00                  _evb_lcd_text
                    0x1a7a                  _get_domain_ip
                    0x1a78                  _get_domain_name
                    0x1a9c                  _http_request
                    0x1a9a                  _http_response
                    0x19c4                  _lease_time
                    0x19cc                  _next_dhcp_time
                    0x19d6                  _pRIPMSG
                    0x1a7e                  _query_data
                    0x19c1                  _retry_count
                    0x1946                  _romfl_list
                    0x19f8                  _sio_head
                    0x19d8                  _sio_rxd
                    0x19fa                  _sio_tail
                    0x1a88                  _sock_flag
                    0x1a90                  _sys_tick_1s
                    0x1a8e                  _sys_tick_5ms
                    0x19fc                  _uart_handler

External Symbols in Program Memory (by address):

                  0x000200                  __resetPRI
                  0x0002d8                  printf.io:_prout
                  0x0002f2                  __iprintf
                  0x000302                  _islower
                  0x00030e                  _toupper
                  0x00031c                  _memset
                  0x00032a                  _puts
                  0x000344                  _strtok
                  0x00037c                  _strcmp
                  0x0003a0                  _strchr
                  0x0003b2                  _strlen
                  0x0003c0                  _strcpy
                  0x0003d0                  _strstr
                  0x0003fa                  _memcpy
                  0x000408                  sprintf.io:_prout
                  0x000414                  __isprintf
                  0x000436                  _memcmp
                  0x000456                  _strcat
                  0x000474                  _fwrite
                  0x00051e                  ___iPrintf
                  0x000690                  _fputs
                  0x00071c                  _fputc
                  0x000768                  _strspn
                  0x00078c                  _strcspn
                  0x0007b0                  __Fwprep
                  0x000836                  _memchr
                  0x00084c                  __DNKfflush
                  0x0008c6                  __Vacopy
                  0x0008d0                  ___iPutfld
                  0x000b58                  __Puttxt
                  0x000cec                  _strrchr
                  0x000d64                  _malloc
                  0x000dbe                  __Closreg
                  0x000dca                  _fclose
                  0x000e4c                  fclose.o:_closeall
                  0x000e64                  __Litob
                  0x000fd2                  __Getmem
                  0x000fe0                  _free
                  0x001046                  __Atexit
                  0x00112e                  ___udivmoddi3
                  0x0011c6                  ___udivdi3
                  0x0011d4                  ___umoddi3
                  0x0011dc                  ___divdi3
                  0x001212                  ___moddi3
                  0x0012d4                  ___muldi3
                  0x001330                  ___umuldi3
                  0x001374                  _loopback_tcps
                  0x0014cc                  _loopback_tcpc
                  0x001638                  _loopback_udp
                  0x00172a                  _strupr
                  0x001762                  _ping_request
                  0x001a50                  _ping_usage
                  0x001a9e                  _web_server
                  0x001be4                  _proc_http
                  0x001e80                  _replace_sys_env_value
                  0x0020cc                  _init_channel_handler
                  0x0020f6                  _register_channel_handler
                  0x00210c                  _unregister_channel_handler
                  0x00212a                  _init_conf_variables
                  0x0021ae                  _set_sysinfo
                  0x0021be                  _get_sysinfo
                  0x002206                  _get_reset_flag
                  0x002216                  _set_reset_flag
                  0x002224                  _get_system_any_port
                  0x00227e                  _set_netconf
                  0x00228e                  _get_netconf
                  0x002316                  _set_chconf
                  0x002326                  _get_chconf
                  0x002382                  _load_factory_netconf
                  0x002396                  _load_factory_chconf
                  0x0023aa                  _display_netconf
                  0x002454                  _display_chconf
                  0x002538                  _evb_init
                  0x00256e                  _evb_soft_reset
                  0x00257e                  _evb_logo
                  0x002616                  _evb_lcd_logo
                  0x00265a                  _evb_get_lcd_text
                  0x00267c                  _evb_set_lcd_text
                  0x0026d8                  _mcu_init
                  0x002726                  _net_init
                  0x00274e                  _LcdCommandW
                  0x002770                  _LcdDataW
                  0x002792                  _lcd_ready
                  0x00279e                  _lcd_ready2
                  0x0027aa                  _lcd_clrscr
                  0x0027b6                  _lcd_init
                  0x0027d8                  _lcd_gotoxy
                  0x002832                  _lcd_puts
                  0x002860                  _lcd_putch
                  0x00286e                  _led_init
                  0x002882                  _led_on
                  0x0028a2                  _sys_led_on
                  0x0028b6                  _led_off
                  0x0028d4                  _sys_led_off
                  0x0028e8                  _led_state
                  0x00290e                  _sys_led_state
                  0x002920                  _led_toggle
                  0x00293a                  _sys_led_toggle
                  0x00294c                  _check_manage
                  0x0029f0                  _manage_config
                  0x002b14                  _manage_network
                  0x002e4e                  _manage_channel
                  0x002f8e                  _select_ch_app
                  0x0033d4                  _InitSEEP
                  0x0033e2                  _i2c_waitForIdle
                  0x00341a                  _i2c_start
                  0x003432                  _i2c_repStart
                  0x00344a                  _i2c_stop
                  0x003462                  _i2c_read
                  0x003486                  _i2c_write
                  0x0034b4                  _eeprom_write_byte
                  0x0034d2                  _eeprom_read_byte
                  0x0034f4                  _eeprom_write_word
                  0x003512                  _eeprom_read_word
                  0x003534                  _eeprom_write_block
                  0x003562                  _eeprom_read_block
                  0x003592                  _FF
                  0x003658                  _GG
                  0x00371e                  _HH
                  0x003790                  _II
                  0x003806                  _md5_init
                  0x003848                  _md5_update
                  0x00397a                  _md5_final
                  0x00464e                  _socket
                  0x00472c                  _close
                  0x004752                  _listen
                  0x00479a                  _connect
                  0x0048c4                  _disconnect
                  0x0048ea                  _send
                  0x0049e8                  _recv
                  0x004a2e                  _sendto
                  0x004bba                  _recvfrom
                  0x004ddc                  _igmpsend
                  0x004e96                  _reset_DHCP_time
                  0x004eb2                  _send_DHCP_DISCOVER
                  0x005168                  _send_DHCP_REQUEST
                  0x005546                  _send_DHCP_RELEASE_DECLINE
                  0x005836                  _parseDHCPMSG
                  0x005abe                  _check_DHCP_state
                  0x005bde                  _check_DHCP_Timeout
                  0x005c4a                  _set_DHCP_network
                  0x005c68                  _check_leasedIP
                  0x005cac                  _getIP_DHCPS
                  0x005ce8                  _DHCP_timer_handler
                  0x005cfa                  _init_dhcp_client
                  0x005d2a                  _proc_ip_conflict
                  0x005d40                  _init_dhcpc_ch
                  0x005dca                  _dns_query
                  0x005f7a                  _dns_makequery
                  0x00609e                  _dns_parse_reponse
                  0x0061be                  _dns_parse_question
                  0x0061f6                  _dns_answer
                  0x0063e8                  _parse_name
                  0x0064ce                  _gethostbyaddr
                  0x006532                  _gethostbyname
                  0x0065a2                  _unescape_http_url
                  0x006622                  _make_http_response_head
                  0x0066a8                  _find_http_uri_type
                  0x00677a                  _parse_http_request
                  0x00681e                  _get_http_param_value
                  0x00689e                  _get_http_uri_name
                  0x0068ea                  _ping
                  0x006c94                  _DisplayPingStatistics
                  0x006d58                  _SendPingReply
                  0x006e02                  _main
                  0x006f44                  _wait_1us
                  0x006f74                  _wait_10ms
                  0x006f88                  _wait_1ms
                  0x006f9c                  _InitPMP
                  0x006fda                  _ReadPMP
                  0x006ffc                  _ReadPMP2
                  0x00701a                  _WritePMP
                  0x00702e                  _FastPMP
                  0x007044                  _SlowPMP
                  0x00705a                  __U1RXInterrupt
                  0x0070a8                  _uart_init
                  0x00711c                  _uart_keyhit
                  0x007144                  _uart0_putchar
                  0x007162                  _uart0_getchar
                  0x00718a                  _write
                  0x0071b2                  _read
                  0x0071e4                  _uart_puts
                  0x007212                  _uart_gets
                  0x007312                  _uart_flush_rx
                  0x00731c                  __T1Interrupt
                  0x00733a                  __T2Interrupt
                  0x007396                  _init_timer
                  0x007446                  _set_timer
                  0x00749a                  _kill_timer
                  0x007510                  _search_file
                  0x00755e                  _inet_ntoa
                  0x0075b2                  _inet_ntoa_pad
                  0x007606                  _inet_addr
                  0x0076b6                  _VerifyIPAddress
                  0x00773a                  _GetDestAddr
                  0x007790                  _GetDestPort
                  0x0077c4                  _htons
                  0x0077d0                  _htonl
                  0x0077dc                  _ntohs
                  0x0077ea                  _ntohl
                  0x0077f6                  _CheckDestInLocal
                  0x007850                  _getSocket
                  0x00788a                  _checksum
                  0x00791e                  _D2C
                  0x00795a                  _C2D
                  0x0079b2                  _ATOI
                  0x0079ec                  _ValidATOI
                  0x007a4c                  _replacetochar
                  0x007a8a                  _swaps
                  0x007aac                  _swapl
                  0x007baa                  _getISR
                  0x007bbc                  _putISR
                  0x007bd0                  _getIINCHIP_RxMAX
                  0x007be2                  _getIINCHIP_TxMAX
                  0x007bf4                  _getIINCHIP_RxMASK
                  0x007c06                  _getIINCHIP_TxMASK
                  0x007c18                  _getIINCHIP_RxBASE
                  0x007c2a                  _getIINCHIP_TxBASE
                  0x007c3c                  _IINCHIP_WRITE
                  0x007c52                  _IINCHIP_READ
                  0x007c66                  _wiz_write_buf
                  0x007c98                  _wiz_read_buf
                  0x007cce                  __INT0Interrupt
                  0x007dd0                  _iinchip_init
                  0x007dda                  _sysinit
                  0x007fd6                  _setMR
                  0x007fe4                  _setGAR
                  0x00800e                  _getGWIP
                  0x00803e                  _setSUBR
                  0x008068                  _setSHAR
                  0x0080a6                  _setSIPR
                  0x0080d0                  _getIR
                  0x0080dc                  _setRTR
                  0x0080f8                  _setRCR
                  0x008106                  _setIMR
                  0x008114                  _getGAR
                  0x008144                  _getSUBR
                  0x008174                  _getSHAR
                  0x0081b8                  _getSIPR
                  0x0081e8                  _getSn_DHAR
                  0x008262                  _setSn_DHAR
                  0x0082e2                  _getSn_DIPR
                  0x008338                  _setSn_DIPR
                  0x008390                  _getSn_DPORT
                  0x0083c2                  _setSn_DPORT
                  0x0083f2                  _setSn_MSS
                  0x008426                  _setSn_TTL
                  0x00843e                  _setSn_PROTO
                  0x008456                  _getSn_IR
                  0x00846c                  _getSn_SR
                  0x008482                  _getSn_TX_FSR
                  0x0084f4                  _getSn_RX_RSR
                  0x008566                  _send_data_processing
                  0x0085da                  _recv_data_processing
                  0x00864e                  _write_data
                  0x0086c2                  _read_data
                  0x00cfbc                  _file0data
                  0x00d8d4                  _file1data
                  0x00dfbe                  _file2data
                  0x00ee10                  _file3data
                  0x00f3bc                  _file4data
                  0x00f490                  _file5data
                  0x00f574                  _file6data
                  0x01043e                  __DefaultInterrupt

External Symbols in Program Memory (by name):

                  0x0079b2                  _ATOI
                  0x00795a                  _C2D
                  0x0077f6                  _CheckDestInLocal
                  0x00791e                  _D2C
                  0x005ce8                  _DHCP_timer_handler
                  0x006c94                  _DisplayPingStatistics
                  0x003592                  _FF
                  0x00702e                  _FastPMP
                  0x003658                  _GG
                  0x00773a                  _GetDestAddr
                  0x007790                  _GetDestPort
                  0x00371e                  _HH
                  0x003790                  _II
                  0x007c52                  _IINCHIP_READ
                  0x007c3c                  _IINCHIP_WRITE
                  0x006f9c                  _InitPMP
                  0x0033d4                  _InitSEEP
                  0x00274e                  _LcdCommandW
                  0x002770                  _LcdDataW
                  0x006fda                  _ReadPMP
                  0x006ffc                  _ReadPMP2
                  0x006d58                  _SendPingReply
                  0x007044                  _SlowPMP
                  0x0079ec                  _ValidATOI
                  0x0076b6                  _VerifyIPAddress
                  0x00701a                  _WritePMP
                  0x001046                  __Atexit
                  0x000dbe                  __Closreg
                  0x00084c                  __DNKfflush
                  0x01043e                  __DefaultInterrupt
                  0x0007b0                  __Fwprep
                  0x000fd2                  __Getmem
                  0x007cce                  __INT0Interrupt
                  0x000e64                  __Litob
                  0x000b58                  __Puttxt
                  0x00731c                  __T1Interrupt
                  0x00733a                  __T2Interrupt
                  0x00705a                  __U1RXInterrupt
                  0x0008c6                  __Vacopy
                  0x0011dc                  ___divdi3
                  0x00051e                  ___iPrintf
                  0x0008d0                  ___iPutfld
                  0x001212                  ___moddi3
                  0x0012d4                  ___muldi3
                  0x0011c6                  ___udivdi3
                  0x00112e                  ___udivmoddi3
                  0x0011d4                  ___umoddi3
                  0x001330                  ___umuldi3
                  0x0002f2                  __iprintf
                  0x000414                  __isprintf
                  0x000200                  __resetPRI
                  0x005bde                  _check_DHCP_Timeout
                  0x005abe                  _check_DHCP_state
                  0x005c68                  _check_leasedIP
                  0x00294c                  _check_manage
                  0x00788a                  _checksum
                  0x00472c                  _close
                  0x00479a                  _connect
                  0x0048c4                  _disconnect
                  0x002454                  _display_chconf
                  0x0023aa                  _display_netconf
                  0x0061f6                  _dns_answer
                  0x005f7a                  _dns_makequery
                  0x0061be                  _dns_parse_question
                  0x00609e                  _dns_parse_reponse
                  0x005dca                  _dns_query
                  0x003562                  _eeprom_read_block
                  0x0034d2                  _eeprom_read_byte
                  0x003512                  _eeprom_read_word
                  0x003534                  _eeprom_write_block
                  0x0034b4                  _eeprom_write_byte
                  0x0034f4                  _eeprom_write_word
                  0x00265a                  _evb_get_lcd_text
                  0x002538                  _evb_init
                  0x002616                  _evb_lcd_logo
                  0x00257e                  _evb_logo
                  0x00267c                  _evb_set_lcd_text
                  0x00256e                  _evb_soft_reset
                  0x000dca                  _fclose
                  0x00cfbc                  _file0data
                  0x00d8d4                  _file1data
                  0x00dfbe                  _file2data
                  0x00ee10                  _file3data
                  0x00f3bc                  _file4data
                  0x00f490                  _file5data
                  0x00f574                  _file6data
                  0x0066a8                  _find_http_uri_type
                  0x00071c                  _fputc
                  0x000690                  _fputs
                  0x000fe0                  _free
                  0x000474                  _fwrite
                  0x008114                  _getGAR
                  0x00800e                  _getGWIP
                  0x007c18                  _getIINCHIP_RxBASE
                  0x007bf4                  _getIINCHIP_RxMASK
                  0x007bd0                  _getIINCHIP_RxMAX
                  0x007c2a                  _getIINCHIP_TxBASE
                  0x007c06                  _getIINCHIP_TxMASK
                  0x007be2                  _getIINCHIP_TxMAX
                  0x005cac                  _getIP_DHCPS
                  0x0080d0                  _getIR
                  0x007baa                  _getISR
                  0x008174                  _getSHAR
                  0x0081b8                  _getSIPR
                  0x008144                  _getSUBR
                  0x0081e8                  _getSn_DHAR
                  0x0082e2                  _getSn_DIPR
                  0x008390                  _getSn_DPORT
                  0x008456                  _getSn_IR
                  0x0084f4                  _getSn_RX_RSR
                  0x00846c                  _getSn_SR
                  0x008482                  _getSn_TX_FSR
                  0x007850                  _getSocket
                  0x002326                  _get_chconf
                  0x00681e                  _get_http_param_value
                  0x00689e                  _get_http_uri_name
                  0x00228e                  _get_netconf
                  0x002206                  _get_reset_flag
                  0x0021be                  _get_sysinfo
                  0x002224                  _get_system_any_port
                  0x0064ce                  _gethostbyaddr
                  0x006532                  _gethostbyname
                  0x0077d0                  _htonl
                  0x0077c4                  _htons
                  0x003462                  _i2c_read
                  0x003432                  _i2c_repStart
                  0x00341a                  _i2c_start
                  0x00344a                  _i2c_stop
                  0x0033e2                  _i2c_waitForIdle
                  0x003486                  _i2c_write
                  0x004ddc                  _igmpsend
                  0x007dd0                  _iinchip_init
                  0x007606                  _inet_addr
                  0x00755e                  _inet_ntoa
                  0x0075b2                  _inet_ntoa_pad
                  0x0020cc                  _init_channel_handler
                  0x00212a                  _init_conf_variables
                  0x005cfa                  _init_dhcp_client
                  0x005d40                  _init_dhcpc_ch
                  0x007396                  _init_timer
                  0x000302                  _islower
                  0x00749a                  _kill_timer
                  0x0027aa                  _lcd_clrscr
                  0x0027d8                  _lcd_gotoxy
                  0x0027b6                  _lcd_init
                  0x002860                  _lcd_putch
                  0x002832                  _lcd_puts
                  0x002792                  _lcd_ready
                  0x00279e                  _lcd_ready2
                  0x00286e                  _led_init
                  0x0028b6                  _led_off
                  0x002882                  _led_on
                  0x0028e8                  _led_state
                  0x002920                  _led_toggle
                  0x004752                  _listen
                  0x002396                  _load_factory_chconf
                  0x002382                  _load_factory_netconf
                  0x0014cc                  _loopback_tcpc
                  0x001374                  _loopback_tcps
                  0x001638                  _loopback_udp
                  0x006e02                  _main
                  0x006622                  _make_http_response_head
                  0x000d64                  _malloc
                  0x002e4e                  _manage_channel
                  0x0029f0                  _manage_config
                  0x002b14                  _manage_network
                  0x0026d8                  _mcu_init
                  0x00397a                  _md5_final
                  0x003806                  _md5_init
                  0x003848                  _md5_update
                  0x000836                  _memchr
                  0x000436                  _memcmp
                  0x0003fa                  _memcpy
                  0x00031c                  _memset
                  0x002726                  _net_init
                  0x0077ea                  _ntohl
                  0x0077dc                  _ntohs
                  0x005836                  _parseDHCPMSG
                  0x00677a                  _parse_http_request
                  0x0063e8                  _parse_name
                  0x0068ea                  _ping
                  0x001762                  _ping_request
                  0x001a50                  _ping_usage
                  0x001be4                  _proc_http
                  0x005d2a                  _proc_ip_conflict
                  0x007bbc                  _putISR
                  0x00032a                  _puts
                  0x0071b2                  _read
                  0x0086c2                  _read_data
                  0x0049e8                  _recv
                  0x0085da                  _recv_data_processing
                  0x004bba                  _recvfrom
                  0x0020f6                  _register_channel_handler
                  0x001e80                  _replace_sys_env_value
                  0x007a4c                  _replacetochar
                  0x004e96                  _reset_DHCP_time
                  0x007510                  _search_file
                  0x002f8e                  _select_ch_app
                  0x0048ea                  _send
                  0x004eb2                  _send_DHCP_DISCOVER
                  0x005546                  _send_DHCP_RELEASE_DECLINE
                  0x005168                  _send_DHCP_REQUEST
                  0x008566                  _send_data_processing
                  0x004a2e                  _sendto
                  0x007fe4                  _setGAR
                  0x008106                  _setIMR
                  0x007fd6                  _setMR
                  0x0080f8                  _setRCR
                  0x0080dc                  _setRTR
                  0x008068                  _setSHAR
                  0x0080a6                  _setSIPR
                  0x00803e                  _setSUBR
                  0x008262                  _setSn_DHAR
                  0x008338                  _setSn_DIPR
                  0x0083c2                  _setSn_DPORT
                  0x0083f2                  _setSn_MSS
                  0x00843e                  _setSn_PROTO
                  0x008426                  _setSn_TTL
                  0x005c4a                  _set_DHCP_network
                  0x002316                  _set_chconf
                  0x00227e                  _set_netconf
                  0x002216                  _set_reset_flag
                  0x0021ae                  _set_sysinfo
                  0x007446                  _set_timer
                  0x00464e                  _socket
                  0x000456                  _strcat
                  0x0003a0                  _strchr
                  0x00037c                  _strcmp
                  0x0003c0                  _strcpy
                  0x00078c                  _strcspn
                  0x0003b2                  _strlen
                  0x000cec                  _strrchr
                  0x000768                  _strspn
                  0x0003d0                  _strstr
                  0x000344                  _strtok
                  0x00172a                  _strupr
                  0x007aac                  _swapl
                  0x007a8a                  _swaps
                  0x0028d4                  _sys_led_off
                  0x0028a2                  _sys_led_on
                  0x00290e                  _sys_led_state
                  0x00293a                  _sys_led_toggle
                  0x007dda                  _sysinit
                  0x00030e                  _toupper
                  0x007162                  _uart0_getchar
                  0x007144                  _uart0_putchar
                  0x007312                  _uart_flush_rx
                  0x007212                  _uart_gets
                  0x0070a8                  _uart_init
                  0x00711c                  _uart_keyhit
                  0x0071e4                  _uart_puts
                  0x0065a2                  _unescape_http_url
                  0x00210c                  _unregister_channel_handler
                  0x006f74                  _wait_10ms
                  0x006f88                  _wait_1ms
                  0x006f44                  _wait_1us
                  0x001a9e                  _web_server
                  0x007c98                  _wiz_read_buf
                  0x007c66                  _wiz_write_buf
                  0x00718a                  _write
                  0x00864e                  _write_data
                  0x000e4c                  fclose.o:_closeall
                  0x0002d8                  printf.io:_prout
                  0x000408                  sprintf.io:_prout

Memory Configuration

Name             Origin             Length             Attributes
data             0x000800           0x002000           a !xr
reset            0x000000           0x000004  
ivt              0x000004           0x0000fc  
aivt             0x000104           0x0000fc  
program          0x000200           0x0155fc           xr
config2          0x0157fc           0x000002  
config1          0x0157fe           0x000002  
*default*        0x000000           0xffffffff  

Linker script and memory map

LOAD loopback.o
LOAD ping_app.o
LOAD webserver.o
LOAD channel.o
LOAD config.o
LOAD evb.o
LOAD lcd.o
LOAD led.o
LOAD manage.o
LOAD SEEP.o
LOAD md5.o
LOAD socket.o
LOAD dhcp.o
LOAD dns.o
LOAD httpd.o
LOAD ping.o
LOAD main.o
LOAD delay.o
LOAD pmp.o
LOAD serial.o
LOAD timer.o
LOAD romfs.o
LOAD searchfile.o
LOAD sockutil.o
LOAD util.o
LOAD w5100.o
                    0x157fc                  __CONFIG2 = 0x157fc
                    0x157fe                  __CONFIG1 = 0x157fe
                    0x0004                  __IVT_BASE = 0x4
                    0x0104                  __AIVT_BASE = 0x104
                    0x0800                  __DATA_BASE = 0x800
                    0x0200                  __CODE_BASE = 0x200

.reset            0x000000          0x4
                  0x000000          0x2 SHORT 0x200 <code 336> (__reset)
                  0x000001          0x2 SHORT 0x4
                  0x000002          0x2 SHORT 0x0 ((<code 336> (__reset) >> 0x10) & 0x7f)
                  0x000003          0x2 SHORT 0x0

.text             0x000200       0x8536
 *(.init)
 .init            0x000200         0x80 c:/program files/microchip/mplab c30/bin/../lib\libpic30-coff.a(crt0.o)
                  0x000200                  _resetPRI
                  0x000200                  _reset
                  0x000214                  _psv_init
                  0x000224                  _data_init
 *(.handle)
 .handle          0x000280         0x58 jump_table
 *(.libc)
 .libc            0x0002d8         0x2a c:/program files/microchip/mplab c30/bin/../lib\libc-coff.a(printf.io)
                  0x0002d8                  printf.io:_prout
                  0x0002f2                  _iprintf
 .libc            0x000302          0xc c:/program files/microchip/mplab c30/bin/../lib\libc-coff.a(islower.os)
                  0x000302                  islower
 .libc            0x00030e          0xe c:/program files/microchip/mplab c30/bin/../lib\libc-coff.a(toupper.os)
                  0x00030e                  toupper
 .libc            0x00031c          0xe c:/program files/microchip/mplab c30/bin/../lib\libc-coff.a(memset.o)
                  0x00031c                  memset
 .libc            0x00032a         0x1a c:/program files/microchip/mplab c30/bin/../lib\libc-coff.a(puts.o)
                  0x00032a                  puts
 .libc            0x000344         0x38 c:/program files/microchip/mplab c30/bin/../lib\libc-coff.a(strtok.o)
                  0x000344                  strtok
 .libc            0x00037c         0x24 c:/program files/microchip/mplab c30/bin/../lib\libc-coff.a(strcmp.o)
                  0x00037c                  strcmp
 .libc            0x0003a0         0x12 c:/program files/microchip/mplab c30/bin/../lib\libc-coff.a(strchr.o)
                  0x0003a0                  strchr
 .libc            0x0003b2          0xe c:/program files/microchip/mplab c30/bin/../lib\libc-coff.a(strlen.o)
                  0x0003b2                  strlen
 .libc            0x0003c0         0x10 c:/program files/microchip/mplab c30/bin/../lib\libc-coff.a(strcpy.o)
                  0x0003c0                  strcpy
 .libc            0x0003d0         0x2a c:/program files/microchip/mplab c30/bin/../lib\libc-coff.a(strstr.o)
                  0x0003d0                  strstr
 .libc            0x0003fa          0xe c:/program files/microchip/mplab c30/bin/../lib\libc-coff.a(memcpy.o)
                  0x0003fa                  memcpy
 .libc            0x000408         0x2e c:/program files/microchip/mplab c30/bin/../lib\libc-coff.a(sprintf.io)
                  0x000408                  sprintf.io:_prout
                  0x000414                  _isprintf
 .libc            0x000436         0x20 c:/program files/microchip/mplab c30/bin/../lib\libc-coff.a(memcmp.o)
                  0x000436                  memcmp
 .libc            0x000456         0x1e c:/program files/microchip/mplab c30/bin/../lib\libc-coff.a(strcat.o)
                  0x000456                  strcat
 .libc            0x000474         0xaa c:/program files/microchip/mplab c30/bin/../lib\libc-coff.a(fwrite.o)
                  0x000474                  fwrite
 .libc            0x00051e        0x172 c:/program files/microchip/mplab c30/bin/../lib\libc-coff.a(xprintf.io)
                  0x00051e                  __iPrintf
 .libc            0x000690         0x8c c:/program files/microchip/mplab c30/bin/../lib\libc-coff.a(fputs.o)
                  0x000690                  fputs
 .libc            0x00071c         0x4c c:/program files/microchip/mplab c30/bin/../lib\libc-coff.a(fputc.o)
                  0x00071c                  fputc
 .libc            0x000768         0x24 c:/program files/microchip/mplab c30/bin/../lib\libc-coff.a(strspn.o)
                  0x000768                  strspn
 .libc            0x00078c         0x24 c:/program files/microchip/mplab c30/bin/../lib\libc-coff.a(strcspn.o)
                  0x00078c                  strcspn
 .libc            0x0007b0         0x86 c:/program files/microchip/mplab c30/bin/../lib\libc-coff.a(xfwprep.o)
                  0x0007b0                  _Fwprep
 .libc            0x000836         0x16 c:/program files/microchip/mplab c30/bin/../lib\libc-coff.a(memchr.o)
                  0x000836                  memchr
 .libc            0x00084c         0x7a c:/program files/microchip/mplab c30/bin/../lib\libc-coff.a(fflush.o)
                  0x00084c                  _DNKfflush
 .libc            0x0008c6          0xa c:/program files/microchip/mplab c30/bin/../lib\libc-coff.a(xvacopy.o)
                  0x0008c6                  _Vacopy
 .libc            0x0008d0        0x288 c:/program files/microchip/mplab c30/bin/../lib\libc-coff.a(xputfld.io)
                  0x0008d0                  __iPutfld
 .libc            0x000b58        0x194 c:/program files/microchip/mplab c30/bin/../lib\libc-coff.a(xputtxt.o)
                  0x000b58                  _Puttxt
 .libc            0x000cec         0x16 c:/program files/microchip/mplab c30/bin/../lib\libc-coff.a(strrchr.o)
                  0x000cec                  strrchr
 .libc            0x000d02         0xb8 c:/program files/microchip/mplab c30/bin/../lib\libc-coff.a(malloc.o)
                  0x000d64                  malloc
 .libc            0x000dba         0xaa c:/program files/microchip/mplab c30/bin/../lib\libc-coff.a(fclose.o)
                  0x000dbe                  _Closreg
                  0x000dca                  fclose
                  0x000e4c                  fclose.o:_closeall
 .libc            0x000e64        0x16e c:/program files/microchip/mplab c30/bin/../lib\libc-coff.a(xlitob.o)
                  0x000e64                  _Litob
 .libc            0x000fd2          0xe c:/program files/microchip/mplab c30/bin/../lib\libc-coff.a(xgetmem.o)
                  0x000fd2                  _Getmem
 .libc            0x000fe0         0x66 c:/program files/microchip/mplab c30/bin/../lib\libc-coff.a(free.o)
                  0x000fe0                  free
 .libc            0x001046         0x1a c:/program files/microchip/mplab c30/bin/../lib\libc-coff.a(xatexit.o)
                  0x001046                  _Atexit
 .libc            0x001060         0x18 c:/program files/microchip/mplab c30/bin/../lib\libpic30-coff.a(remove.o)
                  0x001064                  remove
 .libc            0x001078         0x2c c:/program files/microchip/mplab c30/bin/../lib\libpic30-coff.a(sbrk.o)
                  0x001078                  sbrk
 .libc            0x0010a4         0x1e c:/program files/microchip/mplab c30/bin/../lib\libpic30-coff.a(brk.o)
                  0x0010a4                  brk
 *(.libm)
 .libm            0x0010c2        0x212 c:/program files/microchip/mplab c30/bin/../lib\libm-coff.a(divmoddi3.o)
                  0x00112e                  __udivmoddi3
                  0x0011c6                  __udivdi3
                  0x0011d4                  __umoddi3
                  0x0011dc                  __divdi3
                  0x001212                  __moddi3
 .libm            0x0012d4         0x5c c:/program files/microchip/mplab c30/bin/../lib\libm-coff.a(muldi3.o)
                  0x0012d4                  __muldi3
 .libm            0x001330         0x44 c:/program files/microchip/mplab c30/bin/../lib\libm-coff.a(umuldi3.o)
                  0x001330                  __umuldi3
 *(.libdsp)
 *(.lib*)
 *(.text)
 .text            0x001374        0x3b6 loopback.o
                  0x001374                  loopback_tcps
                  0x0014cc                  loopback_tcpc
                  0x001638                  loopback_udp
 .text            0x00172a        0x374 ping_app.o
                  0x00172a                  strupr
                  0x001762                  ping_request
                  0x001a50                  ping_usage
 .text            0x001a9e        0x62e webserver.o
                  0x001a9e                  web_server
                  0x001be4                  proc_http
                  0x001e80                  replace_sys_env_value
 .text            0x0020cc         0x5e channel.o
                  0x0020cc                  init_channel_handler
                  0x0020f6                  register_channel_handler
                  0x00210c                  unregister_channel_handler
 .text            0x00212a        0x40e config.o
                  0x00212a                  init_conf_variables
                  0x0021ae                  set_sysinfo
                  0x0021be                  get_sysinfo
                  0x002206                  get_reset_flag
                  0x002216                  set_reset_flag
                  0x002224                  get_system_any_port
                  0x00227e                  set_netconf
                  0x00228e                  get_netconf
                  0x002316                  set_chconf
                  0x002326                  get_chconf
                  0x002382                  load_factory_netconf
                  0x002396                  load_factory_chconf
                  0x0023aa                  display_netconf
                  0x002454                  display_chconf
 .text            0x002538        0x216 evb.o
                  0x002538                  evb_init
                  0x00256e                  evb_soft_reset
                  0x00257e                  evb_logo
                  0x002616                  evb_lcd_logo
                  0x00265a                  evb_get_lcd_text
                  0x00267c                  evb_set_lcd_text
                  0x0026d8                  mcu_init
                  0x002726                  net_init
 .text            0x00274e        0x120 lcd.o
                  0x00274e                  LcdCommandW
                  0x002770                  LcdDataW
                  0x002792                  lcd_ready
                  0x00279e                  lcd_ready2
                  0x0027aa                  lcd_clrscr
                  0x0027b6                  lcd_init
                  0x0027d8                  lcd_gotoxy
                  0x002832                  lcd_puts
                  0x002860                  lcd_putch
 .text            0x00286e         0xde led.o
                  0x00286e                  led_init
                  0x002882                  led_on
                  0x0028a2                  sys_led_on
                  0x0028b6                  led_off
                  0x0028d4                  sys_led_off
                  0x0028e8                  led_state
                  0x00290e                  sys_led_state
                  0x002920                  led_toggle
                  0x00293a                  sys_led_toggle
 .text            0x00294c        0xa88 manage.o
                  0x00294c                  check_manage
                  0x0029f0                  manage_config
                  0x002b14                  manage_network
                  0x002e4e                  manage_channel
                  0x002f8e                  select_ch_app
 .text            0x0033d4        0x1be SEEP.o
                  0x0033d4                  InitSEEP
                  0x0033e2                  i2c_waitForIdle
                  0x00341a                  i2c_start
                  0x003432                  i2c_repStart
                  0x00344a                  i2c_stop
                  0x003462                  i2c_read
                  0x003486                  i2c_write
                  0x0034b4                  eeprom_write_byte
                  0x0034d2                  eeprom_read_byte
                  0x0034f4                  eeprom_write_word
                  0x003512                  eeprom_read_word
                  0x003534                  eeprom_write_block
                  0x003562                  eeprom_read_block
 .text            0x003592       0x10bc md5.o
                  0x003592                  FF
                  0x003658                  GG
                  0x00371e                  HH
                  0x003790                  II
                  0x003806                  md5_init
                  0x003848                  md5_update
                  0x00397a                  md5_final
 .text            0x00464e        0x848 socket.o
                  0x00464e                  socket
                  0x00472c                  close
                  0x004752                  listen
                  0x00479a                  connect
                  0x0048c4                  disconnect
                  0x0048ea                  send
                  0x0049e8                  recv
                  0x004a2e                  sendto
                  0x004bba                  recvfrom
                  0x004ddc                  igmpsend
 .text            0x004e96        0xf34 dhcp.o
                  0x004e96                  reset_DHCP_time
                  0x004eb2                  send_DHCP_DISCOVER
                  0x005168                  send_DHCP_REQUEST
                  0x005546                  send_DHCP_RELEASE_DECLINE
                  0x005836                  parseDHCPMSG
                  0x005abe                  check_DHCP_state
                  0x005bde                  check_DHCP_Timeout
                  0x005c4a                  set_DHCP_network
                  0x005c68                  check_leasedIP
                  0x005cac                  getIP_DHCPS
                  0x005ce8                  DHCP_timer_handler
                  0x005cfa                  init_dhcp_client
                  0x005d2a                  proc_ip_conflict
                  0x005d40                  init_dhcpc_ch
 .text            0x005dca        0x7d8 dns.o
                  0x005dca                  dns_query
                  0x005f7a                  dns_makequery
                  0x00609e                  dns_parse_reponse
                  0x0061be                  dns_parse_question
                  0x0061f6                  dns_answer
                  0x0063e8                  parse_name
                  0x0064ce                  gethostbyaddr
                  0x006532                  gethostbyname
 .text            0x0065a2        0x348 httpd.o
                  0x0065a2                  unescape_http_url
                  0x006622                  make_http_response_head
                  0x0066a8                  find_http_uri_type
                  0x00677a                  parse_http_request
                  0x00681e                  get_http_param_value
                  0x00689e                  get_http_uri_name
 .text            0x0068ea        0x518 ping.o
                  0x0068ea                  ping
                  0x006c94                  DisplayPingStatistics
                  0x006d58                  SendPingReply
 .text            0x006e02        0x142 main.o
                  0x006e02                  main
 .text            0x006f44         0x58 delay.o
                  0x006f44                  wait_1us
                  0x006f74                  wait_10ms
                  0x006f88                  wait_1ms
 .text            0x006f9c         0xbe pmp.o
                  0x006f9c                  InitPMP
                  0x006fda                  ReadPMP
                  0x006ffc                  ReadPMP2
                  0x00701a                  WritePMP
                  0x00702e                  FastPMP
                  0x007044                  SlowPMP
 .text            0x00705a        0x2c2 serial.o
                  0x00705a                  _U1RXInterrupt
                  0x0070a8                  uart_init
                  0x00711c                  uart_keyhit
                  0x007144                  uart0_putchar
                  0x007162                  uart0_getchar
                  0x00718a                  write
                  0x0071b2                  read
                  0x0071e4                  uart_puts
                  0x007212                  uart_gets
                  0x007312                  uart_flush_rx
 .text            0x00731c        0x1f4 timer.o
                  0x00731c                  _T1Interrupt
                  0x00733a                  _T2Interrupt
                  0x007396                  init_timer
                  0x007446                  set_timer
                  0x00749a                  kill_timer
 .text            0x007510         0x4e searchfile.o
                  0x007510                  search_file
 .text            0x00755e        0x3c0 sockutil.o
                  0x00755e                  inet_ntoa
                  0x0075b2                  inet_ntoa_pad
                  0x007606                  inet_addr
                  0x0076b6                  VerifyIPAddress
                  0x00773a                  GetDestAddr
                  0x007790                  GetDestPort
                  0x0077c4                  htons
                  0x0077d0                  htonl
                  0x0077dc                  ntohs
                  0x0077ea                  ntohl
                  0x0077f6                  CheckDestInLocal
                  0x007850                  getSocket
                  0x00788a                  checksum
 .text            0x00791e        0x28c util.o
                  0x00791e                  D2C
                  0x00795a                  C2D
                  0x0079b2                  ATOI
                  0x0079ec                  ValidATOI
                  0x007a4c                  replacetochar
                  0x007a8a                  swaps
                  0x007aac                  swapl
 .text            0x007baa        0xb8c w5100.o
                  0x007baa                  getISR
                  0x007bbc                  putISR
                  0x007bd0                  getIINCHIP_RxMAX
                  0x007be2                  getIINCHIP_TxMAX
                  0x007bf4                  getIINCHIP_RxMASK
                  0x007c06                  getIINCHIP_TxMASK
                  0x007c18                  getIINCHIP_RxBASE
                  0x007c2a                  getIINCHIP_TxBASE
                  0x007c3c                  IINCHIP_WRITE
                  0x007c52                  IINCHIP_READ
                  0x007c66                  wiz_write_buf
                  0x007c98                  wiz_read_buf
                  0x007cce                  _INT0Interrupt
                  0x007dd0                  iinchip_init
                  0x007dda                  sysinit
                  0x007fd6                  setMR
                  0x007fe4                  setGAR
                  0x00800e                  getGWIP
                  0x00803e                  setSUBR
                  0x008068                  setSHAR
                  0x0080a6                  setSIPR
                  0x0080d0                  getIR
                  0x0080dc                  setRTR
                  0x0080f8                  setRCR
                  0x008106                  setIMR
                  0x008114                  getGAR
                  0x008144                  getSUBR
                  0x008174                  getSHAR
                  0x0081b8                  getSIPR
                  0x0081e8                  getSn_DHAR
                  0x008262                  setSn_DHAR
                  0x0082e2                  getSn_DIPR
                  0x008338                  setSn_DIPR
                  0x008390                  getSn_DPORT
                  0x0083c2                  setSn_DPORT
                  0x0083f2                  setSn_MSS
                  0x008426                  setSn_TTL
                  0x00843e                  setSn_PROTO
                  0x008456                  getSn_IR
                  0x00846c                  getSn_SR
                  0x008482                  getSn_TX_FSR
                  0x0084f4                  getSn_RX_RSR
                  0x008566                  send_data_processing
                  0x0085da                  recv_data_processing
                  0x00864e                  write_data
                  0x0086c2                  read_data

__CONFIG2
 *(__CONFIG2.sec)

__CONFIG1
 *(__CONFIG1.sec)

.comment          0x000000         0x5e
 *(.comment)
 .comment         0x000000         0x5e c:/program files/microchip/mplab c30/bin/../lib\libc-coff.a(xfiles.o)

.debug_info
 *(.debug_info)
 *(.gnu.linkonce.wi.*)

.debug_abbrev
 *(.debug_abbrev)

.debug_line
 *(.debug_line)

.debug_frame
 *(.debug_frame)

.debug_str
 *(.debug_str)

.debug_loc
 *(.debug_loc)

.debug_macinfo
 *(.debug_macinfo)

.debug_pubnames
 *(.debug_pubnames)

.debug_ranges
 *(.debug_ranges)

.debug_aranges
 *(.debug_aranges)

.ivt              0x000004         0xfc
                  0x000004          0x4 LONG 0x1043e DEFINED (__ReservedTrap0)?<code 336> (__ReservedTrap0):<code 336> (__DefaultInterrupt)
                  0x000006          0x4 LONG 0x1043e DEFINED (__OscillatorFail)?<code 336> (__OscillatorFail):<code 336> (__DefaultInterrupt)
                  0x000008          0x4 LONG 0x1043e DEFINED (__AddressError)?<code 336> (__AddressError):<code 336> (__DefaultInterrupt)
                  0x00000a          0x4 LONG 0x1043e DEFINED (__StackError)?<code 336> (__StackError):<code 336> (__DefaultInterrupt)
                  0x00000c          0x4 LONG 0x1043e DEFINED (__MathError)?<code 336> (__MathError):<code 336> (__DefaultInterrupt)
                  0x00000e          0x4 LONG 0x1043e DEFINED (__ReservedTrap5)?<code 336> (__ReservedTrap5):<code 336> (__DefaultInterrupt)
                  0x000010          0x4 LONG 0x1043e DEFINED (__ReservedTrap6)?<code 336> (__ReservedTrap6):<code 336> (__DefaultInterrupt)
                  0x000012          0x4 LONG 0x1043e DEFINED (__ReservedTrap7)?<code 336> (__ReservedTrap7):<code 336> (__DefaultInterrupt)
                  0x000014          0x4 LONG 0x7cce DEFINED (__INT0Interrupt)?<code 336> (__INT0Interrupt):<code 336> (__DefaultInterrupt)
                  0x000016          0x4 LONG 0x1043e DEFINED (__IC1Interrupt)?<code 336> (__IC1Interrupt):<code 336> (__DefaultInterrupt)
                  0x000018          0x4 LONG 0x1043e DEFINED (__OC1Interrupt)?<code 336> (__OC1Interrupt):<code 336> (__DefaultInterrupt)
                  0x00001a          0x4 LONG 0x731c DEFINED (__T1Interrupt)?<code 336> (__T1Interrupt):<code 336> (__DefaultInterrupt)
                  0x00001c          0x4 LONG 0x1043e DEFINED (__Interrupt4)?<code 336> (__Interrupt4):<code 336> (__DefaultInterrupt)
                  0x00001e          0x4 LONG 0x1043e DEFINED (__IC2Interrupt)?<code 336> (__IC2Interrupt):<code 336> (__DefaultInterrupt)
                  0x000020          0x4 LONG 0x1043e DEFINED (__OC2Interrupt)?<code 336> (__OC2Interrupt):<code 336> (__DefaultInterrupt)
                  0x000022          0x4 LONG 0x733a DEFINED (__T2Interrupt)?<code 336> (__T2Interrupt):<code 336> (__DefaultInterrupt)
                  0x000024          0x4 LONG 0x1043e DEFINED (__T3Interrupt)?<code 336> (__T3Interrupt):<code 336> (__DefaultInterrupt)
                  0x000026          0x4 LONG 0x1043e DEFINED (__SPI1ErrInterrupt)?<code 336> (__SPI1ErrInterrupt):<code 336> (__DefaultInterrupt)
                  0x000028          0x4 LONG 0x1043e DEFINED (__SPI1Interrupt)?<code 336> (__SPI1Interrupt):<code 336> (__DefaultInterrupt)
                  0x00002a          0x4 LONG 0x705a DEFINED (__U1RXInterrupt)?<code 336> (__U1RXInterrupt):<code 336> (__DefaultInterrupt)
                  0x00002c          0x4 LONG 0x1043e DEFINED (__U1TXInterrupt)?<code 336> (__U1TXInterrupt):<code 336> (__DefaultInterrupt)
                  0x00002e          0x4 LONG 0x1043e DEFINED (__ADC1Interrupt)?<code 336> (__ADC1Interrupt):<code 336> (__DefaultInterrupt)
                  0x000030          0x4 LONG 0x1043e DEFINED (__Interrupt14)?<code 336> (__Interrupt14):<code 336> (__DefaultInterrupt)
                  0x000032          0x4 LONG 0x1043e DEFINED (__Interrupt15)?<code 336> (__Interrupt15):<code 336> (__DefaultInterrupt)
                  0x000034          0x4 LONG 0x1043e DEFINED (__SI2C1Interrupt)?<code 336> (__SI2C1Interrupt):<code 336> (__DefaultInterrupt)
                  0x000036          0x4 LONG 0x1043e DEFINED (__MI2C1Interrupt)?<code 336> (__MI2C1Interrupt):<code 336> (__DefaultInterrupt)
                  0x000038          0x4 LONG 0x1043e DEFINED (__CompInterrupt)?<code 336> (__CompInterrupt):<code 336> (__DefaultInterrupt)
                  0x00003a          0x4 LONG 0x1043e DEFINED (__CNInterrupt)?<code 336> (__CNInterrupt):<code 336> (__DefaultInterrupt)
                  0x00003c          0x4 LONG 0x1043e DEFINED (__INT1Interrupt)?<code 336> (__INT1Interrupt):<code 336> (__DefaultInterrupt)
                  0x00003e          0x4 LONG 0x1043e DEFINED (__Interrupt21)?<code 336> (__Interrupt21):<code 336> (__DefaultInterrupt)
                  0x000040          0x4 LONG 0x1043e DEFINED (__Interrupt22)?<code 336> (__Interrupt22):<code 336> (__DefaultInterrupt)
                  0x000042          0x4 LONG 0x1043e DEFINED (__Interrupt23)?<code 336> (__Interrupt23):<code 336> (__DefaultInterrupt)
                  0x000044          0x4 LONG 0x1043e DEFINED (__Interrupt24)?<code 336> (__Interrupt24):<code 336> (__DefaultInterrupt)
                  0x000046          0x4 LONG 0x1043e DEFINED (__OC3Interrupt)?<code 336> (__OC3Interrupt):<code 336> (__DefaultInterrupt)
                  0x000048          0x4 LONG 0x1043e DEFINED (__OC4Interrupt)?<code 336> (__OC4Interrupt):<code 336> (__DefaultInterrupt)
                  0x00004a          0x4 LONG 0x1043e DEFINED (__T4Interrupt)?<code 336> (__T4Interrupt):<code 336> (__DefaultInterrupt)
                  0x00004c          0x4 LONG 0x1043e DEFINED (__T5Interrupt)?<code 336> (__T5Interrupt):<code 336> (__DefaultInterrupt)
                  0x00004e          0x4 LONG 0x1043e DEFINED (__INT2Interrupt)?<code 336> (__INT2Interrupt):<code 336> (__DefaultInterrupt)
                  0x000050          0x4 LONG 0x1043e DEFINED (__U2RXInterrupt)?<code 336> (__U2RXInterrupt):<code 336> (__DefaultInterrupt)
                  0x000052          0x4 LONG 0x1043e DEFINED (__U2TXInterrupt)?<code 336> (__U2TXInterrupt):<code 336> (__DefaultInterrupt)
                  0x000054          0x4 LONG 0x1043e DEFINED (__SPI2ErrInterrupt)?<code 336> (__SPI2ErrInterrupt):<code 336> (__DefaultInterrupt)
                  0x000056          0x4 LONG 0x1043e DEFINED (__SPI2Interrupt)?<code 336> (__SPI2Interrupt):<code 336> (__DefaultInterrupt)
                  0x000058          0x4 LONG 0x1043e DEFINED (__Interrupt34)?<code 336> (__Interrupt34):<code 336> (__DefaultInterrupt)
                  0x00005a          0x4 LONG 0x1043e DEFINED (__Interrupt35)?<code 336> (__Interrupt35):<code 336> (__DefaultInterrupt)
                  0x00005c          0x4 LONG 0x1043e DEFINED (__Interrupt36)?<code 336> (__Interrupt36):<code 336> (__DefaultInterrupt)
                  0x00005e          0x4 LONG 0x1043e DEFINED (__IC3Interrupt)?<code 336> (__IC3Interrupt):<code 336> (__DefaultInterrupt)
                  0x000060          0x4 LONG 0x1043e DEFINED (__IC4Interrupt)?<code 336> (__IC4Interrupt):<code 336> (__DefaultInterrupt)
                  0x000062          0x4 LONG 0x1043e DEFINED (__IC5Interrupt)?<code 336> (__IC5Interrupt):<code 336> (__DefaultInterrupt)
                  0x000064          0x4 LONG 0x1043e DEFINED (__Interrupt40)?<code 336> (__Interrupt40):<code 336> (__DefaultInterrupt)
                  0x000066          0x4 LONG 0x1043e DEFINED (__OC5Interrupt)?<code 336> (__OC5Interrupt):<code 336> (__DefaultInterrupt)
                  0x000068          0x4 LONG 0x1043e DEFINED (__Interrupt42)?<code 336> (__Interrupt42):<code 336> (__DefaultInterrupt)
                  0x00006a          0x4 LONG 0x1043e DEFINED (__Interrupt43)?<code 336> (__Interrupt43):<code 336> (__DefaultInterrupt)
                  0x00006c          0x4 LONG 0x1043e DEFINED (__Interrupt44)?<code 336> (__Interrupt44):<code 336> (__DefaultInterrupt)
                  0x00006e          0x4 LONG 0x1043e DEFINED (__PMPInterrupt)?<code 336> (__PMPInterrupt):<code 336> (__DefaultInterrupt)
                  0x000070          0x4 LONG 0x1043e DEFINED (__Interrupt46)?<code 336> (__Interrupt46):<code 336> (__DefaultInterrupt)
                  0x000072          0x4 LONG 0x1043e DEFINED (__Interrupt47)?<code 336> (__Interrupt47):<code 336> (__DefaultInterrupt)
                  0x000074          0x4 LONG 0x1043e DEFINED (__Interrupt48)?<code 336> (__Interrupt48):<code 336> (__DefaultInterrupt)
                  0x000076          0x4 LONG 0x1043e DEFINED (__SI2C2Interrupt)?<code 336> (__SI2C2Interrupt):<code 336> (__DefaultInterrupt)
                  0x000078          0x4 LONG 0x1043e DEFINED (__MI2C2Interrupt)?<code 336> (__MI2C2Interrupt):<code 336> (__DefaultInterrupt)
                  0x00007a          0x4 LONG 0x1043e DEFINED (__Interrupt51)?<code 336> (__Interrupt51):<code 336> (__DefaultInterrupt)
                  0x00007c          0x4 LONG 0x1043e DEFINED (__Interrupt52)?<code 336> (__Interrupt52):<code 336> (__DefaultInterrupt)
                  0x00007e          0x4 LONG 0x1043e DEFINED (__INT3Interrupt)?<code 336> (__INT3Interrupt):<code 336> (__DefaultInterrupt)
                  0x000080          0x4 LONG 0x1043e DEFINED (__INT4Interrupt)?<code 336> (__INT4Interrupt):<code 336> (__DefaultInterrupt)
                  0x000082          0x4 LONG 0x1043e DEFINED (__Interrupt55)?<code 336> (__Interrupt55):<code 336> (__DefaultInterrupt)
                  0x000084          0x4 LONG 0x1043e DEFINED (__Interrupt56)?<code 336> (__Interrupt56):<code 336> (__DefaultInterrupt)
                  0x000086          0x4 LONG 0x1043e DEFINED (__Interrupt57)?<code 336> (__Interrupt57):<code 336> (__DefaultInterrupt)
                  0x000088          0x4 LONG 0x1043e DEFINED (__Interrupt58)?<code 336> (__Interrupt58):<code 336> (__DefaultInterrupt)
                  0x00008a          0x4 LONG 0x1043e DEFINED (__Interrupt59)?<code 336> (__Interrupt59):<code 336> (__DefaultInterrupt)
                  0x00008c          0x4 LONG 0x1043e DEFINED (__Interrupt60)?<code 336> (__Interrupt60):<code 336> (__DefaultInterrupt)
                  0x00008e          0x4 LONG 0x1043e DEFINED (__Interrupt61)?<code 336> (__Interrupt61):<code 336> (__DefaultInterrupt)
                  0x000090          0x4 LONG 0x1043e DEFINED (__RTCCInterrupt)?<code 336> (__RTCCInterrupt):<code 336> (__DefaultInterrupt)
                  0x000092          0x4 LONG 0x1043e DEFINED (__Interrupt63)?<code 336> (__Interrupt63):<code 336> (__DefaultInterrupt)
                  0x000094          0x4 LONG 0x1043e DEFINED (__Interrupt64)?<code 336> (__Interrupt64):<code 336> (__DefaultInterrupt)
                  0x000096          0x4 LONG 0x1043e DEFINED (__U1ErrInterrupt)?<code 336> (__U1ErrInterrupt):<code 336> (__DefaultInterrupt)
                  0x000098          0x4 LONG 0x1043e DEFINED (__U2ErrInterrupt)?<code 336> (__U2ErrInterrupt):<code 336> (__DefaultInterrupt)
                  0x00009a          0x4 LONG 0x1043e DEFINED (__CRCInterrupt)?<code 336> (__CRCInterrupt):<code 336> (__DefaultInterrupt)
                  0x00009c          0x4 LONG 0x1043e DEFINED (__Interrupt68)?<code 336> (__Interrupt68):<code 336> (__DefaultInterrupt)
                  0x00009e          0x4 LONG 0x1043e DEFINED (__Interrupt69)?<code 336> (__Interrupt69):<code 336> (__DefaultInterrupt)
                  0x0000a0          0x4 LONG 0x1043e DEFINED (__Interrupt70)?<code 336> (__Interrupt70):<code 336> (__DefaultInterrupt)
                  0x0000a2          0x4 LONG 0x1043e DEFINED (__Interrupt71)?<code 336> (__Interrupt71):<code 336> (__DefaultInterrupt)
                  0x0000a4          0x4 LONG 0x1043e DEFINED (__Interrupt72)?<code 336> (__Interrupt72):<code 336> (__DefaultInterrupt)
                  0x0000a6          0x4 LONG 0x1043e DEFINED (__Interrupt73)?<code 336> (__Interrupt73):<code 336> (__DefaultInterrupt)
                  0x0000a8          0x4 LONG 0x1043e DEFINED (__Interrupt74)?<code 336> (__Interrupt74):<code 336> (__DefaultInterrupt)
                  0x0000aa          0x4 LONG 0x1043e DEFINED (__Interrupt75)?<code 336> (__Interrupt75):<code 336> (__DefaultInterrupt)
                  0x0000ac          0x4 LONG 0x1043e DEFINED (__Interrupt76)?<code 336> (__Interrupt76):<code 336> (__DefaultInterrupt)
                  0x0000ae          0x4 LONG 0x1043e DEFINED (__Interrupt77)?<code 336> (__Interrupt77):<code 336> (__DefaultInterrupt)
                  0x0000b0          0x4 LONG 0x1043e DEFINED (__Interrupt78)?<code 336> (__Interrupt78):<code 336> (__DefaultInterrupt)
                  0x0000b2          0x4 LONG 0x1043e DEFINED (__Interrupt79)?<code 336> (__Interrupt79):<code 336> (__DefaultInterrupt)
                  0x0000b4          0x4 LONG 0x1043e DEFINED (__Interrupt80)?<code 336> (__Interrupt80):<code 336> (__DefaultInterrupt)
                  0x0000b6          0x4 LONG 0x1043e DEFINED (__Interrupt81)?<code 336> (__Interrupt81):<code 336> (__DefaultInterrupt)
                  0x0000b8          0x4 LONG 0x1043e DEFINED (__Interrupt82)?<code 336> (__Interrupt82):<code 336> (__DefaultInterrupt)
                  0x0000ba          0x4 LONG 0x1043e DEFINED (__Interrupt83)?<code 336> (__Interrupt83):<code 336> (__DefaultInterrupt)
                  0x0000bc          0x4 LONG 0x1043e DEFINED (__Interrupt84)?<code 336> (__Interrupt84):<code 336> (__DefaultInterrupt)
                  0x0000be          0x4 LONG 0x1043e DEFINED (__Interrupt85)?<code 336> (__Interrupt85):<code 336> (__DefaultInterrupt)
                  0x0000c0          0x4 LONG 0x1043e DEFINED (__Interrupt86)?<code 336> (__Interrupt86):<code 336> (__DefaultInterrupt)
                  0x0000c2          0x4 LONG 0x1043e DEFINED (__Interrupt87)?<code 336> (__Interrupt87):<code 336> (__DefaultInterrupt)
                  0x0000c4          0x4 LONG 0x1043e DEFINED (__Interrupt88)?<code 336> (__Interrupt88):<code 336> (__DefaultInterrupt)
                  0x0000c6          0x4 LONG 0x1043e DEFINED (__Interrupt89)?<code 336> (__Interrupt89):<code 336> (__DefaultInterrupt)
                  0x0000c8          0x4 LONG 0x1043e DEFINED (__Interrupt90)?<code 336> (__Interrupt90):<code 336> (__DefaultInterrupt)
                  0x0000ca          0x4 LONG 0x1043e DEFINED (__Interrupt91)?<code 336> (__Interrupt91):<code 336> (__DefaultInterrupt)
                  0x0000cc          0x4 LONG 0x1043e DEFINED (__Interrupt92)?<code 336> (__Interrupt92):<code 336> (__DefaultInterrupt)
                  0x0000ce          0x4 LONG 0x1043e DEFINED (__Interrupt93)?<code 336> (__Interrupt93):<code 336> (__DefaultInterrupt)
                  0x0000d0          0x4 LONG 0x1043e DEFINED (__Interrupt94)?<code 336> (__Interrupt94):<code 336> (__DefaultInterrupt)
                  0x0000d2          0x4 LONG 0x1043e DEFINED (__Interrupt95)?<code 336> (__Interrupt95):<code 336> (__DefaultInterrupt)
                  0x0000d4          0x4 LONG 0x1043e DEFINED (__Interrupt96)?<code 336> (__Interrupt96):<code 336> (__DefaultInterrupt)
                  0x0000d6          0x4 LONG 0x1043e DEFINED (__Interrupt97)?<code 336> (__Interrupt97):<code 336> (__DefaultInterrupt)
                  0x0000d8          0x4 LONG 0x1043e DEFINED (__Interrupt98)?<code 336> (__Interrupt98):<code 336> (__DefaultInterrupt)
                  0x0000da          0x4 LONG 0x1043e DEFINED (__Interrupt99)?<code 336> (__Interrupt99):<code 336> (__DefaultInterrupt)
                  0x0000dc          0x4 LONG 0x1043e DEFINED (__Interrupt100)?<code 336> (__Interrupt100):<code 336> (__DefaultInterrupt)
                  0x0000de          0x4 LONG 0x1043e DEFINED (__Interrupt101)?<code 336> (__Interrupt101):<code 336> (__DefaultInterrupt)
                  0x0000e0          0x4 LONG 0x1043e DEFINED (__Interrupt102)?<code 336> (__Interrupt102):<code 336> (__DefaultInterrupt)
                  0x0000e2          0x4 LONG 0x1043e DEFINED (__Interrupt103)?<code 336> (__Interrupt103):<code 336> (__DefaultInterrupt)
                  0x0000e4          0x4 LONG 0x1043e DEFINED (__Interrupt104)?<code 336> (__Interrupt104):<code 336> (__DefaultInterrupt)
                  0x0000e6          0x4 LONG 0x1043e DEFINED (__Interrupt105)?<code 336> (__Interrupt105):<code 336> (__DefaultInterrupt)
                  0x0000e8          0x4 LONG 0x1043e DEFINED (__Interrupt106)?<code 336> (__Interrupt106):<code 336> (__DefaultInterrupt)
                  0x0000ea          0x4 LONG 0x1043e DEFINED (__Interrupt107)?<code 336> (__Interrupt107):<code 336> (__DefaultInterrupt)
                  0x0000ec          0x4 LONG 0x1043e DEFINED (__Interrupt108)?<code 336> (__Interrupt108):<code 336> (__DefaultInterrupt)
                  0x0000ee          0x4 LONG 0x1043e DEFINED (__Interrupt109)?<code 336> (__Interrupt109):<code 336> (__DefaultInterrupt)
                  0x0000f0          0x4 LONG 0x1043e DEFINED (__Interrupt110)?<code 336> (__Interrupt110):<code 336> (__DefaultInterrupt)
                  0x0000f2          0x4 LONG 0x1043e DEFINED (__Interrupt111)?<code 336> (__Interrupt111):<code 336> (__DefaultInterrupt)
                  0x0000f4          0x4 LONG 0x1043e DEFINED (__Interrupt112)?<code 336> (__Interrupt112):<code 336> (__DefaultInterrupt)
                  0x0000f6          0x4 LONG 0x1043e DEFINED (__Interrupt113)?<code 336> (__Interrupt113):<code 336> (__DefaultInterrupt)
                  0x0000f8          0x4 LONG 0x1043e DEFINED (__Interrupt114)?<code 336> (__Interrupt114):<code 336> (__DefaultInterrupt)
                  0x0000fa          0x4 LONG 0x1043e DEFINED (__Interrupt115)?<code 336> (__Interrupt115):<code 336> (__DefaultInterrupt)
                  0x0000fc          0x4 LONG 0x1043e DEFINED (__Interrupt116)?<code 336> (__Interrupt116):<code 336> (__DefaultInterrupt)
                  0x0000fe          0x4 LONG 0x1043e DEFINED (__Interrupt117)?<code 336> (__Interrupt117):<code 336> (__DefaultInterrupt)

.aivt             0x000104         0xfc
                  0x000104          0x4 LONG 0x1043e DEFINED (__AltReservedTrap0)?<code 336> (__AltReservedTrap0):DEFINED (__ReservedTrap0)?<code 336> (__ReservedTrap0):<code 336> (__DefaultInterrupt)
                  0x000106          0x4 LONG 0x1043e DEFINED (__AltOscillatorFail)?<code 336> (__AltOscillatorFail):DEFINED (__OscillatorFail)?<code 336> (__OscillatorFail):<code 336> (__DefaultInterrupt)
                  0x000108          0x4 LONG 0x1043e DEFINED (__AltAddressError)?<code 336> (__AltAddressError):DEFINED (__AddressError)?<code 336> (__AddressError):<code 336> (__DefaultInterrupt)
                  0x00010a          0x4 LONG 0x1043e DEFINED (__AltStackError)?<code 336> (__AltStackError):DEFINED (__StackError)?<code 336> (__StackError):<code 336> (__DefaultInterrupt)
                  0x00010c          0x4 LONG 0x1043e DEFINED (__AltMathError)?<code 336> (__AltMathError):DEFINED (__MathError)?<code 336> (__MathError):<code 336> (__DefaultInterrupt)
                  0x00010e          0x4 LONG 0x1043e DEFINED (__AltReservedTrap5)?<code 336> (__AltReservedTrap5):DEFINED (__ReservedTrap5)?<code 336> (__ReservedTrap5):<code 336> (__DefaultInterrupt)
                  0x000110          0x4 LONG 0x1043e DEFINED (__AltReservedTrap6)?<code 336> (__AltReservedTrap6):DEFINED (__ReservedTrap6)?<code 336> (__ReservedTrap6):<code 336> (__DefaultInterrupt)
                  0x000112          0x4 LONG 0x1043e DEFINED (__AltReservedTrap7)?<code 336> (__AltReservedTrap7):DEFINED (__ReservedTrap7)?<code 336> (__ReservedTrap7):<code 336> (__DefaultInterrupt)
                  0x000114          0x4 LONG 0x7cce DEFINED (__AltINT0Interrupt)?<code 336> (__AltINT0Interrupt):DEFINED (__INT0Interrupt)?<code 336> (__INT0Interrupt):<code 336> (__DefaultInterrupt)
                  0x000116          0x4 LONG 0x1043e DEFINED (__AltIC1Interrupt)?<code 336> (__AltIC1Interrupt):DEFINED (__IC1Interrupt)?<code 336> (__IC1Interrupt):<code 336> (__DefaultInterrupt)
                  0x000118          0x4 LONG 0x1043e DEFINED (__AltOC1Interrupt)?<code 336> (__AltOC1Interrupt):DEFINED (__OC1Interrupt)?<code 336> (__OC1Interrupt):<code 336> (__DefaultInterrupt)
                  0x00011a          0x4 LONG 0x731c DEFINED (__AltT1Interrupt)?<code 336> (__AltT1Interrupt):DEFINED (__T1Interrupt)?<code 336> (__T1Interrupt):<code 336> (__DefaultInterrupt)
                  0x00011c          0x4 LONG 0x1043e DEFINED (__AltInterrupt4)?<code 336> (__AltInterrupt4):DEFINED (__Interrupt4)?<code 336> (__Interrupt4):<code 336> (__DefaultInterrupt)
                  0x00011e          0x4 LONG 0x1043e DEFINED (__AltIC2Interrupt)?<code 336> (__AltIC2Interrupt):DEFINED (__IC2Interrupt)?<code 336> (__IC2Interrupt):<code 336> (__DefaultInterrupt)
                  0x000120          0x4 LONG 0x1043e DEFINED (__AltOC2Interrupt)?<code 336> (__AltOC2Interrupt):DEFINED (__OC2Interrupt)?<code 336> (__OC2Interrupt):<code 336> (__DefaultInterrupt)
                  0x000122          0x4 LONG 0x733a DEFINED (__AltT2Interrupt)?<code 336> (__AltT2Interrupt):DEFINED (__T2Interrupt)?<code 336> (__T2Interrupt):<code 336> (__DefaultInterrupt)
                  0x000124          0x4 LONG 0x1043e DEFINED (__AltT3Interrupt)?<code 336> (__AltT3Interrupt):DEFINED (__T3Interrupt)?<code 336> (__T3Interrupt):<code 336> (__DefaultInterrupt)
                  0x000126          0x4 LONG 0x1043e DEFINED (__AltSPI1ErrInterrupt)?<code 336> (__AltSPI1ErrInterrupt):DEFINED (__SPI1ErrInterrupt)?<code 336> (__SPI1ErrInterrupt):<code 336> (__DefaultInterrupt)
                  0x000128          0x4 LONG 0x1043e DEFINED (__AltSPI1Interrupt)?<code 336> (__AltSPI1Interrupt):DEFINED (__SPI1Interrupt)?<code 336> (__SPI1Interrupt):<code 336> (__DefaultInterrupt)
                  0x00012a          0x4 LONG 0x705a DEFINED (__AltU1RXInterrupt)?<code 336> (__AltU1RXInterrupt):DEFINED (__U1RXInterrupt)?<code 336> (__U1RXInterrupt):<code 336> (__DefaultInterrupt)
                  0x00012c          0x4 LONG 0x1043e DEFINED (__AltU1TXInterrupt)?<code 336> (__AltU1TXInterrupt):DEFINED (__U1TXInterrupt)?<code 336> (__U1TXInterrupt):<code 336> (__DefaultInterrupt)
                  0x00012e          0x4 LONG 0x1043e DEFINED (__AltADC1Interrupt)?<code 336> (__AltADC1Interrupt):DEFINED (__ADC1Interrupt)?<code 336> (__ADC1Interrupt):<code 336> (__DefaultInterrupt)
                  0x000130          0x4 LONG 0x1043e DEFINED (__AltInterrupt14)?<code 336> (__AltInterrupt14):DEFINED (__Interrupt14)?<code 336> (__Interrupt14):<code 336> (__DefaultInterrupt)
                  0x000132          0x4 LONG 0x1043e DEFINED (__AltInterrupt15)?<code 336> (__AltInterrupt15):DEFINED (__Interrupt15)?<code 336> (__Interrupt15):<code 336> (__DefaultInterrupt)
                  0x000134          0x4 LONG 0x1043e DEFINED (__AltSI2C1Interrupt)?<code 336> (__AltSI2C1Interrupt):DEFINED (__SI2C1Interrupt)?<code 336> (__SI2C1Interrupt):<code 336> (__DefaultInterrupt)
                  0x000136          0x4 LONG 0x1043e DEFINED (__AltMI2C1Interrupt)?<code 336> (__AltMI2C1Interrupt):DEFINED (__MI2C1Interrupt)?<code 336> (__MI2C1Interrupt):<code 336> (__DefaultInterrupt)
                  0x000138          0x4 LONG 0x1043e DEFINED (__AltCompInterrupt)?<code 336> (__AltCompInterrupt):DEFINED (__CompInterrupt)?<code 336> (__CompInterrupt):<code 336> (__DefaultInterrupt)
                  0x00013a          0x4 LONG 0x1043e DEFINED (__AltCNInterrupt)?<code 336> (__AltCNInterrupt):DEFINED (__CNInterrupt)?<code 336> (__CNInterrupt):<code 336> (__DefaultInterrupt)
                  0x00013c          0x4 LONG 0x1043e DEFINED (__AltINT1Interrupt)?<code 336> (__AltINT1Interrupt):DEFINED (__INT1Interrupt)?<code 336> (__INT1Interrupt):<code 336> (__DefaultInterrupt)
                  0x00013e          0x4 LONG 0x1043e DEFINED (__AltInterrupt21)?<code 336> (__AltInterrupt21):DEFINED (__Interrupt21)?<code 336> (__Interrupt21):<code 336> (__DefaultInterrupt)
                  0x000140          0x4 LONG 0x1043e DEFINED (__AltInterrupt22)?<code 336> (__AltInterrupt22):DEFINED (__Interrupt22)?<code 336> (__Interrupt22):<code 336> (__DefaultInterrupt)
                  0x000142          0x4 LONG 0x1043e DEFINED (__AltInterrupt23)?<code 336> (__AltInterrupt23):DEFINED (__Interrupt23)?<code 336> (__Interrupt23):<code 336> (__DefaultInterrupt)
                  0x000144          0x4 LONG 0x1043e DEFINED (__AltInterrupt24)?<code 336> (__AltInterrupt24):DEFINED (__Interrupt24)?<code 336> (__Interrupt24):<code 336> (__DefaultInterrupt)
                  0x000146          0x4 LONG 0x1043e DEFINED (__AltOC3Interrupt)?<code 336> (__AltOC3Interrupt):DEFINED (__OC3Interrupt)?<code 336> (__OC3Interrupt):<code 336> (__DefaultInterrupt)
                  0x000148          0x4 LONG 0x1043e DEFINED (__AltOC4Interrupt)?<code 336> (__AltOC4Interrupt):DEFINED (__OC4Interrupt)?<code 336> (__OC4Interrupt):<code 336> (__DefaultInterrupt)
                  0x00014a          0x4 LONG 0x1043e DEFINED (__AltT4Interrupt)?<code 336> (__AltT4Interrupt):DEFINED (__T4Interrupt)?<code 336> (__T4Interrupt):<code 336> (__DefaultInterrupt)
                  0x00014c          0x4 LONG 0x1043e DEFINED (__AltT5Interrupt)?<code 336> (__AltT5Interrupt):DEFINED (__T5Interrupt)?<code 336> (__T5Interrupt):<code 336> (__DefaultInterrupt)
                  0x00014e          0x4 LONG 0x1043e DEFINED (__AltINT2Interrupt)?<code 336> (__AltINT2Interrupt):DEFINED (__INT2Interrupt)?<code 336> (__INT2Interrupt):<code 336> (__DefaultInterrupt)
                  0x000150          0x4 LONG 0x1043e DEFINED (__AltU2RXInterrupt)?<code 336> (__AltU2RXInterrupt):DEFINED (__U2RXInterrupt)?<code 336> (__U2RXInterrupt):<code 336> (__DefaultInterrupt)
                  0x000152          0x4 LONG 0x1043e DEFINED (__AltU2TXInterrupt)?<code 336> (__AltU2TXInterrupt):DEFINED (__U2TXInterrupt)?<code 336> (__U2TXInterrupt):<code 336> (__DefaultInterrupt)
                  0x000154          0x4 LONG 0x1043e DEFINED (__AltSPI2ErrInterrupt)?<code 336> (__AltSPI2ErrInterrupt):DEFINED (__SPI2ErrInterrupt)?<code 336> (__SPI2ErrInterrupt):<code 336> (__DefaultInterrupt)
                  0x000156          0x4 LONG 0x1043e DEFINED (__AltSPI2Interrupt)?<code 336> (__AltSPI2Interrupt):DEFINED (__SPI2Interrupt)?<code 336> (__SPI2Interrupt):<code 336> (__DefaultInterrupt)
                  0x000158          0x4 LONG 0x1043e DEFINED (__AltInterrupt34)?<code 336> (__AltInterrupt34):DEFINED (__Interrupt34)?<code 336> (__Interrupt34):<code 336> (__DefaultInterrupt)
                  0x00015a          0x4 LONG 0x1043e DEFINED (__AltInterrupt35)?<code 336> (__AltInterrupt35):DEFINED (__Interrupt35)?<code 336> (__Interrupt35):<code 336> (__DefaultInterrupt)
                  0x00015c          0x4 LONG 0x1043e DEFINED (__AltInterrupt36)?<code 336> (__AltInterrupt36):DEFINED (__Interrupt36)?<code 336> (__Interrupt36):<code 336> (__DefaultInterrupt)
                  0x00015e          0x4 LONG 0x1043e DEFINED (__AltIC3Interrupt)?<code 336> (__AltIC3Interrupt):DEFINED (__IC3Interrupt)?<code 336> (__IC3Interrupt):<code 336> (__DefaultInterrupt)
                  0x000160          0x4 LONG 0x1043e DEFINED (__AltIC4Interrupt)?<code 336> (__AltIC4Interrupt):DEFINED (__IC4Interrupt)?<code 336> (__IC4Interrupt):<code 336> (__DefaultInterrupt)
                  0x000162          0x4 LONG 0x1043e DEFINED (__AltIC5Interrupt)?<code 336> (__AltIC5Interrupt):DEFINED (__IC5Interrupt)?<code 336> (__IC5Interrupt):<code 336> (__DefaultInterrupt)
                  0x000164          0x4 LONG 0x1043e DEFINED (__AltInterrupt40)?<code 336> (__AltInterrupt40):DEFINED (__Interrupt40)?<code 336> (__Interrupt40):<code 336> (__DefaultInterrupt)
                  0x000166          0x4 LONG 0x1043e DEFINED (__AltOC5Interrupt)?<code 336> (__AltOC5Interrupt):DEFINED (__OC5Interrupt)?<code 336> (__OC5Interrupt):<code 336> (__DefaultInterrupt)
                  0x000168          0x4 LONG 0x1043e DEFINED (__AltInterrupt42)?<code 336> (__AltInterrupt42):DEFINED (__Interrupt42)?<code 336> (__Interrupt42):<code 336> (__DefaultInterrupt)
                  0x00016a          0x4 LONG 0x1043e DEFINED (__AltInterrupt43)?<code 336> (__AltInterrupt43):DEFINED (__Interrupt43)?<code 336> (__Interrupt43):<code 336> (__DefaultInterrupt)
                  0x00016c          0x4 LONG 0x1043e DEFINED (__AltInterrupt44)?<code 336> (__AltInterrupt44):DEFINED (__Interrupt44)?<code 336> (__Interrupt44):<code 336> (__DefaultInterrupt)
                  0x00016e          0x4 LONG 0x1043e DEFINED (__AltPMPInterrupt)?<code 336> (__AltPMPInterrupt):DEFINED (__PMPInterrupt)?<code 336> (__PMPInterrupt):<code 336> (__DefaultInterrupt)
                  0x000170          0x4 LONG 0x1043e DEFINED (__AltInterrupt46)?<code 336> (__AltInterrupt46):DEFINED (__Interrupt46)?<code 336> (__Interrupt46):<code 336> (__DefaultInterrupt)
                  0x000172          0x4 LONG 0x1043e DEFINED (__AltInterrupt47)?<code 336> (__AltInterrupt47):DEFINED (__Interrupt47)?<code 336> (__Interrupt47):<code 336> (__DefaultInterrupt)
                  0x000174          0x4 LONG 0x1043e DEFINED (__AltInterrupt48)?<code 336> (__AltInterrupt48):DEFINED (__Interrupt48)?<code 336> (__Interrupt48):<code 336> (__DefaultInterrupt)
                  0x000176          0x4 LONG 0x1043e DEFINED (__AltSI2C2Interrupt)?<code 336> (__AltSI2C2Interrupt):DEFINED (__SI2C2Interrupt)?<code 336> (__SI2C2Interrupt):<code 336> (__DefaultInterrupt)
                  0x000178          0x4 LONG 0x1043e DEFINED (__AltMI2C2Interrupt)?<code 336> (__AltMI2C2Interrupt):DEFINED (__MI2C2Interrupt)?<code 336> (__MI2C2Interrupt):<code 336> (__DefaultInterrupt)
                  0x00017a          0x4 LONG 0x1043e DEFINED (__AltInterrupt51)?<code 336> (__AltInterrupt51):DEFINED (__Interrupt51)?<code 336> (__Interrupt51):<code 336> (__DefaultInterrupt)
                  0x00017c          0x4 LONG 0x1043e DEFINED (__AltInterrupt52)?<code 336> (__AltInterrupt52):DEFINED (__Interrupt52)?<code 336> (__Interrupt52):<code 336> (__DefaultInterrupt)
                  0x00017e          0x4 LONG 0x1043e DEFINED (__AltINT3Interrupt)?<code 336> (__AltINT3Interrupt):DEFINED (__INT3Interrupt)?<code 336> (__INT3Interrupt):<code 336> (__DefaultInterrupt)
                  0x000180          0x4 LONG 0x1043e DEFINED (__AltINT4Interrupt)?<code 336> (__AltINT4Interrupt):DEFINED (__INT4Interrupt)?<code 336> (__INT4Interrupt):<code 336> (__DefaultInterrupt)
                  0x000182          0x4 LONG 0x1043e DEFINED (__AltInterrupt55)?<code 336> (__AltInterrupt55):DEFINED (__Interrupt55)?<code 336> (__Interrupt55):<code 336> (__DefaultInterrupt)
                  0x000184          0x4 LONG 0x1043e DEFINED (__AltInterrupt56)?<code 336> (__AltInterrupt56):DEFINED (__Interrupt56)?<code 336> (__Interrupt56):<code 336> (__DefaultInterrupt)
                  0x000186          0x4 LONG 0x1043e DEFINED (__AltInterrupt57)?<code 336> (__AltInterrupt57):DEFINED (__Interrupt57)?<code 336> (__Interrupt57):<code 336> (__DefaultInterrupt)
                  0x000188          0x4 LONG 0x1043e DEFINED (__AltInterrupt58)?<code 336> (__AltInterrupt58):DEFINED (__Interrupt58)?<code 336> (__Interrupt58):<code 336> (__DefaultInterrupt)
                  0x00018a          0x4 LONG 0x1043e DEFINED (__AltInterrupt59)?<code 336> (__AltInterrupt59):DEFINED (__Interrupt59)?<code 336> (__Interrupt59):<code 336> (__DefaultInterrupt)
                  0x00018c          0x4 LONG 0x1043e DEFINED (__AltInterrupt60)?<code 336> (__AltInterrupt60):DEFINED (__Interrupt60)?<code 336> (__Interrupt60):<code 336> (__DefaultInterrupt)
                  0x00018e          0x4 LONG 0x1043e DEFINED (__AltInterrupt61)?<code 336> (__AltInterrupt61):DEFINED (__Interrupt61)?<code 336> (__Interrupt61):<code 336> (__DefaultInterrupt)
                  0x000190          0x4 LONG 0x1043e DEFINED (__AltRTCCInterrupt)?<code 336> (__AltRTCCInterrupt):DEFINED (__RTCCInterrupt)?<code 336> (__RTCCInterrupt):<code 336> (__DefaultInterrupt)
                  0x000192          0x4 LONG 0x1043e DEFINED (__AltInterrupt63)?<code 336> (__AltInterrupt63):DEFINED (__Interrupt63)?<code 336> (__Interrupt63):<code 336> (__DefaultInterrupt)
                  0x000194          0x4 LONG 0x1043e DEFINED (__AltInterrupt64)?<code 336> (__AltInterrupt64):DEFINED (__Interrupt64)?<code 336> (__Interrupt64):<code 336> (__DefaultInterrupt)
                  0x000196          0x4 LONG 0x1043e DEFINED (__AltU1ErrInterrupt)?<code 336> (__AltU1ErrInterrupt):DEFINED (__U1ErrInterrupt)?<code 336> (__U1ErrInterrupt):<code 336> (__DefaultInterrupt)
                  0x000198          0x4 LONG 0x1043e DEFINED (__AltU2ErrInterrupt)?<code 336> (__AltU2ErrInterrupt):DEFINED (__U2ErrInterrupt)?<code 336> (__U2ErrInterrupt):<code 336> (__DefaultInterrupt)
                  0x00019a          0x4 LONG 0x1043e DEFINED (__AltCRCInterrupt)?<code 336> (__AltCRCInterrupt):DEFINED (__CRCInterrupt)?<code 336> (__CRCInterrupt):<code 336> (__DefaultInterrupt)
                  0x00019c          0x4 LONG 0x1043e DEFINED (__AltInterrupt68)?<code 336> (__AltInterrupt68):DEFINED (__Interrupt68)?<code 336> (__Interrupt68):<code 336> (__DefaultInterrupt)
                  0x00019e          0x4 LONG 0x1043e DEFINED (__AltInterrupt69)?<code 336> (__AltInterrupt69):DEFINED (__Interrupt69)?<code 336> (__Interrupt69):<code 336> (__DefaultInterrupt)
                  0x0001a0          0x4 LONG 0x1043e DEFINED (__AltInterrupt70)?<code 336> (__AltInterrupt70):DEFINED (__Interrupt70)?<code 336> (__Interrupt70):<code 336> (__DefaultInterrupt)
                  0x0001a2          0x4 LONG 0x1043e DEFINED (__AltInterrupt71)?<code 336> (__AltInterrupt71):DEFINED (__Interrupt71)?<code 336> (__Interrupt71):<code 336> (__DefaultInterrupt)
                  0x0001a4          0x4 LONG 0x1043e DEFINED (__AltInterrupt72)?<code 336> (__AltInterrupt72):DEFINED (__Interrupt72)?<code 336> (__Interrupt72):<code 336> (__DefaultInterrupt)
                  0x0001a6          0x4 LONG 0x1043e DEFINED (__AltInterrupt73)?<code 336> (__AltInterrupt73):DEFINED (__Interrupt73)?<code 336> (__Interrupt73):<code 336> (__DefaultInterrupt)
                  0x0001a8          0x4 LONG 0x1043e DEFINED (__AltInterrupt74)?<code 336> (__AltInterrupt74):DEFINED (__Interrupt74)?<code 336> (__Interrupt74):<code 336> (__DefaultInterrupt)
                  0x0001aa          0x4 LONG 0x1043e DEFINED (__AltInterrupt75)?<code 336> (__AltInterrupt75):DEFINED (__Interrupt75)?<code 336> (__Interrupt75):<code 336> (__DefaultInterrupt)
                  0x0001ac          0x4 LONG 0x1043e DEFINED (__AltInterrupt76)?<code 336> (__AltInterrupt76):DEFINED (__Interrupt76)?<code 336> (__Interrupt76):<code 336> (__DefaultInterrupt)
                  0x0001ae          0x4 LONG 0x1043e DEFINED (__AltInterrupt77)?<code 336> (__AltInterrupt77):DEFINED (__Interrupt77)?<code 336> (__Interrupt77):<code 336> (__DefaultInterrupt)
                  0x0001b0          0x4 LONG 0x1043e DEFINED (__AltInterrupt78)?<code 336> (__AltInterrupt78):DEFINED (__Interrupt78)?<code 336> (__Interrupt78):<code 336> (__DefaultInterrupt)
                  0x0001b2          0x4 LONG 0x1043e DEFINED (__AltInterrupt79)?<code 336> (__AltInterrupt79):DEFINED (__Interrupt79)?<code 336> (__Interrupt79):<code 336> (__DefaultInterrupt)
                  0x0001b4          0x4 LONG 0x1043e DEFINED (__AltInterrupt80)?<code 336> (__AltInterrupt80):DEFINED (__Interrupt80)?<code 336> (__Interrupt80):<code 336> (__DefaultInterrupt)
                  0x0001b6          0x4 LONG 0x1043e DEFINED (__AltInterrupt81)?<code 336> (__AltInterrupt81):DEFINED (__Interrupt81)?<code 336> (__Interrupt81):<code 336> (__DefaultInterrupt)
                  0x0001b8          0x4 LONG 0x1043e DEFINED (__AltInterrupt82)?<code 336> (__AltInterrupt82):DEFINED (__Interrupt82)?<code 336> (__Interrupt82):<code 336> (__DefaultInterrupt)
                  0x0001ba          0x4 LONG 0x1043e DEFINED (__AltInterrupt83)?<code 336> (__AltInterrupt83):DEFINED (__Interrupt83)?<code 336> (__Interrupt83):<code 336> (__DefaultInterrupt)
                  0x0001bc          0x4 LONG 0x1043e DEFINED (__AltInterrupt84)?<code 336> (__AltInterrupt84):DEFINED (__Interrupt84)?<code 336> (__Interrupt84):<code 336> (__DefaultInterrupt)
                  0x0001be          0x4 LONG 0x1043e DEFINED (__AltInterrupt85)?<code 336> (__AltInterrupt85):DEFINED (__Interrupt85)?<code 336> (__Interrupt85):<code 336> (__DefaultInterrupt)
                  0x0001c0          0x4 LONG 0x1043e DEFINED (__AltInterrupt86)?<code 336> (__AltInterrupt86):DEFINED (__Interrupt86)?<code 336> (__Interrupt86):<code 336> (__DefaultInterrupt)
                  0x0001c2          0x4 LONG 0x1043e DEFINED (__AltInterrupt87)?<code 336> (__AltInterrupt87):DEFINED (__Interrupt87)?<code 336> (__Interrupt87):<code 336> (__DefaultInterrupt)
                  0x0001c4          0x4 LONG 0x1043e DEFINED (__AltInterrupt88)?<code 336> (__AltInterrupt88):DEFINED (__Interrupt88)?<code 336> (__Interrupt88):<code 336> (__DefaultInterrupt)
                  0x0001c6          0x4 LONG 0x1043e DEFINED (__AltInterrupt89)?<code 336> (__AltInterrupt89):DEFINED (__Interrupt89)?<code 336> (__Interrupt89):<code 336> (__DefaultInterrupt)
                  0x0001c8          0x4 LONG 0x1043e DEFINED (__AltInterrupt90)?<code 336> (__AltInterrupt90):DEFINED (__Interrupt90)?<code 336> (__Interrupt90):<code 336> (__DefaultInterrupt)
                  0x0001ca          0x4 LONG 0x1043e DEFINED (__AltInterrupt91)?<code 336> (__AltInterrupt91):DEFINED (__Interrupt91)?<code 336> (__Interrupt91):<code 336> (__DefaultInterrupt)
                  0x0001cc          0x4 LONG 0x1043e DEFINED (__AltInterrupt92)?<code 336> (__AltInterrupt92):DEFINED (__Interrupt92)?<code 336> (__Interrupt92):<code 336> (__DefaultInterrupt)
                  0x0001ce          0x4 LONG 0x1043e DEFINED (__AltInterrupt93)?<code 336> (__AltInterrupt93):DEFINED (__Interrupt93)?<code 336> (__Interrupt93):<code 336> (__DefaultInterrupt)
                  0x0001d0          0x4 LONG 0x1043e DEFINED (__AltInterrupt94)?<code 336> (__AltInterrupt94):DEFINED (__Interrupt94)?<code 336> (__Interrupt94):<code 336> (__DefaultInterrupt)
                  0x0001d2          0x4 LONG 0x1043e DEFINED (__AltInterrupt95)?<code 336> (__AltInterrupt95):DEFINED (__Interrupt95)?<code 336> (__Interrupt95):<code 336> (__DefaultInterrupt)
                  0x0001d4          0x4 LONG 0x1043e DEFINED (__AltInterrupt96)?<code 336> (__AltInterrupt96):DEFINED (__Interrupt96)?<code 336> (__Interrupt96):<code 336> (__DefaultInterrupt)
                  0x0001d6          0x4 LONG 0x1043e DEFINED (__AltInterrupt97)?<code 336> (__AltInterrupt97):DEFINED (__Interrupt97)?<code 336> (__Interrupt97):<code 336> (__DefaultInterrupt)
                  0x0001d8          0x4 LONG 0x1043e DEFINED (__AltInterrupt98)?<code 336> (__AltInterrupt98):DEFINED (__Interrupt98)?<code 336> (__Interrupt98):<code 336> (__DefaultInterrupt)
                  0x0001da          0x4 LONG 0x1043e DEFINED (__AltInterrupt99)?<code 336> (__AltInterrupt99):DEFINED (__Interrupt99)?<code 336> (__Interrupt99):<code 336> (__DefaultInterrupt)
                  0x0001dc          0x4 LONG 0x1043e DEFINED (__AltInterrupt100)?<code 336> (__AltInterrupt100):DEFINED (__Interrupt100)?<code 336> (__Interrupt100):<code 336> (__DefaultInterrupt)
                  0x0001de          0x4 LONG 0x1043e DEFINED (__AltInterrupt101)?<code 336> (__AltInterrupt101):DEFINED (__Interrupt101)?<code 336> (__Interrupt101):<code 336> (__DefaultInterrupt)
                  0x0001e0          0x4 LONG 0x1043e DEFINED (__AltInterrupt102)?<code 336> (__AltInterrupt102):DEFINED (__Interrupt102)?<code 336> (__Interrupt102):<code 336> (__DefaultInterrupt)
                  0x0001e2          0x4 LONG 0x1043e DEFINED (__AltInterrupt103)?<code 336> (__AltInterrupt103):DEFINED (__Interrupt103)?<code 336> (__Interrupt103):<code 336> (__DefaultInterrupt)
                  0x0001e4          0x4 LONG 0x1043e DEFINED (__AltInterrupt104)?<code 336> (__AltInterrupt104):DEFINED (__Interrupt104)?<code 336> (__Interrupt104):<code 336> (__DefaultInterrupt)
                  0x0001e6          0x4 LONG 0x1043e DEFINED (__AltInterrupt105)?<code 336> (__AltInterrupt105):DEFINED (__Interrupt105)?<code 336> (__Interrupt105):<code 336> (__DefaultInterrupt)
                  0x0001e8          0x4 LONG 0x1043e DEFINED (__AltInterrupt106)?<code 336> (__AltInterrupt106):DEFINED (__Interrupt106)?<code 336> (__Interrupt106):<code 336> (__DefaultInterrupt)
                  0x0001ea          0x4 LONG 0x1043e DEFINED (__AltInterrupt107)?<code 336> (__AltInterrupt107):DEFINED (__Interrupt107)?<code 336> (__Interrupt107):<code 336> (__DefaultInterrupt)
                  0x0001ec          0x4 LONG 0x1043e DEFINED (__AltInterrupt108)?<code 336> (__AltInterrupt108):DEFINED (__Interrupt108)?<code 336> (__Interrupt108):<code 336> (__DefaultInterrupt)
                  0x0001ee          0x4 LONG 0x1043e DEFINED (__AltInterrupt109)?<code 336> (__AltInterrupt109):DEFINED (__Interrupt109)?<code 336> (__Interrupt109):<code 336> (__DefaultInterrupt)
                  0x0001f0          0x4 LONG 0x1043e DEFINED (__AltInterrupt110)?<code 336> (__AltInterrupt110):DEFINED (__Interrupt110)?<code 336> (__Interrupt110):<code 336> (__DefaultInterrupt)
                  0x0001f2          0x4 LONG 0x1043e DEFINED (__AltInterrupt111)?<code 336> (__AltInterrupt111):DEFINED (__Interrupt111)?<code 336> (__Interrupt111):<code 336> (__DefaultInterrupt)
                  0x0001f4          0x4 LONG 0x1043e DEFINED (__AltInterrupt112)?<code 336> (__AltInterrupt112):DEFINED (__Interrupt112)?<code 336> (__Interrupt112):<code 336> (__DefaultInterrupt)
                  0x0001f6          0x4 LONG 0x1043e DEFINED (__AltInterrupt113)?<code 336> (__AltInterrupt113):DEFINED (__Interrupt113)?<code 336> (__Interrupt113):<code 336> (__DefaultInterrupt)
                  0x0001f8          0x4 LONG 0x1043e DEFINED (__AltInterrupt114)?<code 336> (__AltInterrupt114):DEFINED (__Interrupt114)?<code 336> (__Interrupt114):<code 336> (__DefaultInterrupt)
                  0x0001fa          0x4 LONG 0x1043e DEFINED (__AltInterrupt115)?<code 336> (__AltInterrupt115):DEFINED (__Interrupt115)?<code 336> (__Interrupt115):<code 336> (__DefaultInterrupt)
                  0x0001fc          0x4 LONG 0x1043e DEFINED (__AltInterrupt116)?<code 336> (__AltInterrupt116):DEFINED (__Interrupt116)?<code 336> (__Interrupt116):<code 336> (__DefaultInterrupt)
                  0x0001fe          0x4 LONG 0x1043e DEFINED (__AltInterrupt117)?<code 336> (__AltInterrupt117):DEFINED (__Interrupt117)?<code 336> (__Interrupt117):<code 336> (__DefaultInterrupt)
                    0x0000                  WREG0 = 0x0
                    0x0000                  _WREG0 = 0x0
                    0x0002                  WREG1 = 0x2
                    0x0002                  _WREG1 = 0x2
                    0x0004                  WREG2 = 0x4
                    0x0004                  _WREG2 = 0x4
                    0x0006                  WREG3 = 0x6
                    0x0006                  _WREG3 = 0x6
                    0x0008                  WREG4 = 0x8
                    0x0008                  _WREG4 = 0x8
                    0x000a                  WREG5 = 0xa
                    0x000a                  _WREG5 = 0xa
                    0x000c                  WREG6 = 0xc
                    0x000c                  _WREG6 = 0xc
                    0x000e                  WREG7 = 0xe
                    0x000e                  _WREG7 = 0xe
                    0x0010                  WREG8 = 0x10
                    0x0010                  _WREG8 = 0x10
                    0x0012                  WREG9 = 0x12
                    0x0012                  _WREG9 = 0x12
                    0x0014                  WREG10 = 0x14
                    0x0014                  _WREG10 = 0x14
                    0x0016                  WREG11 = 0x16
                    0x0016                  _WREG11 = 0x16
                    0x0018                  WREG12 = 0x18
                    0x0018                  _WREG12 = 0x18
                    0x001a                  WREG13 = 0x1a
                    0x001a                  _WREG13 = 0x1a
                    0x001c                  WREG14 = 0x1c
                    0x001c                  _WREG14 = 0x1c
                    0x001e                  WREG15 = 0x1e
                    0x001e                  _WREG15 = 0x1e
                    0x0020                  SPLIM = 0x20
                    0x0020                  _SPLIM = 0x20
                    0x002e                  PCL = 0x2e
                    0x002e                  _PCL = 0x2e
                    0x0030                  PCH = 0x30
                    0x0030                  _PCH = 0x30
                    0x0032                  TBLPAG = 0x32
                    0x0032                  _TBLPAG = 0x32
                    0x0034                  PSVPAG = 0x34
                    0x0034                  _PSVPAG = 0x34
                    0x0036                  RCOUNT = 0x36
                    0x0036                  _RCOUNT = 0x36
                    0x0042                  SR = 0x42
                    0x0042                  _SR = 0x42
                    0x0042                  _SRbits = 0x42
                    0x0044                  CORCON = 0x44
                    0x0044                  _CORCON = 0x44
                    0x0044                  _CORCONbits = 0x44
                    0x0052                  DISICNT = 0x52
                    0x0052                  _DISICNT = 0x52
                    0x0060                  CNEN1 = 0x60
                    0x0060                  _CNEN1 = 0x60
                    0x0060                  _CNEN1bits = 0x60
                    0x0062                  CNEN2 = 0x62
                    0x0062                  _CNEN2 = 0x62
                    0x0062                  _CNEN2bits = 0x62
                    0x0068                  CNPU1 = 0x68
                    0x0068                  _CNPU1 = 0x68
                    0x0068                  _CNPU1bits = 0x68
                    0x006a                  CNPU2 = 0x6a
                    0x006a                  _CNPU2 = 0x6a
                    0x006a                  _CNPU2bits = 0x6a
                    0x0080                  INTCON1 = 0x80
                    0x0080                  _INTCON1 = 0x80
                    0x0080                  _INTCON1bits = 0x80
                    0x0082                  INTCON2 = 0x82
                    0x0082                  _INTCON2 = 0x82
                    0x0082                  _INTCON2bits = 0x82
                    0x0084                  IFS0 = 0x84
                    0x0084                  _IFS0 = 0x84
                    0x0084                  _IFS0bits = 0x84
                    0x0086                  IFS1 = 0x86
                    0x0086                  _IFS1 = 0x86
                    0x0086                  _IFS1bits = 0x86
                    0x0088                  IFS2 = 0x88
                    0x0088                  _IFS2 = 0x88
                    0x0088                  _IFS2bits = 0x88
                    0x008a                  IFS3 = 0x8a
                    0x008a                  _IFS3 = 0x8a
                    0x008a                  _IFS3bits = 0x8a
                    0x008c                  IFS4 = 0x8c
                    0x008c                  _IFS4 = 0x8c
                    0x008c                  _IFS4bits = 0x8c
                    0x0094                  IEC0 = 0x94
                    0x0094                  _IEC0 = 0x94
                    0x0094                  _IEC0bits = 0x94
                    0x0096                  IEC1 = 0x96
                    0x0096                  _IEC1 = 0x96
                    0x0096                  _IEC1bits = 0x96
                    0x0098                  IEC2 = 0x98
                    0x0098                  _IEC2 = 0x98
                    0x0098                  _IEC2bits = 0x98
                    0x009a                  IEC3 = 0x9a
                    0x009a                  _IEC3 = 0x9a
                    0x009a                  _IEC3bits = 0x9a
                    0x009c                  IEC4 = 0x9c
                    0x009c                  _IEC4 = 0x9c
                    0x009c                  _IEC4bits = 0x9c
                    0x00a4                  IPC0 = 0xa4
                    0x00a4                  _IPC0 = 0xa4
                    0x00a4                  _IPC0bits = 0xa4
                    0x00a6                  IPC1 = 0xa6
                    0x00a6                  _IPC1 = 0xa6
                    0x00a6                  _IPC1bits = 0xa6
                    0x00a8                  IPC2 = 0xa8
                    0x00a8                  _IPC2 = 0xa8
                    0x00a8                  _IPC2bits = 0xa8
                    0x00aa                  IPC3 = 0xaa
                    0x00aa                  _IPC3 = 0xaa
                    0x00aa                  _IPC3bits = 0xaa
                    0x00ac                  IPC4 = 0xac
                    0x00ac                  _IPC4 = 0xac
                    0x00ac                  _IPC4bits = 0xac
                    0x00ae                  IPC5 = 0xae
                    0x00ae                  _IPC5 = 0xae
                    0x00ae                  _IPC5bits = 0xae
                    0x00b0                  IPC6 = 0xb0
                    0x00b0                  _IPC6 = 0xb0
                    0x00b0                  _IPC6bits = 0xb0
                    0x00b2                  IPC7 = 0xb2
                    0x00b2                  _IPC7 = 0xb2
                    0x00b2                  _IPC7bits = 0xb2
                    0x00b4                  IPC8 = 0xb4
                    0x00b4                  _IPC8 = 0xb4
                    0x00b4                  _IPC8bits = 0xb4
                    0x00b6                  IPC9 = 0xb6
                    0x00b6                  _IPC9 = 0xb6
                    0x00b6                  _IPC9bits = 0xb6
                    0x00b8                  IPC10 = 0xb8
                    0x00b8                  _IPC10 = 0xb8
                    0x00b8                  _IPC10bits = 0xb8
                    0x00ba                  IPC11 = 0xba
                    0x00ba                  _IPC11 = 0xba
                    0x00ba                  _IPC11bits = 0xba
                    0x00bc                  IPC12 = 0xbc
                    0x00bc                  _IPC12 = 0xbc
                    0x00bc                  _IPC12bits = 0xbc
                    0x00be                  IPC13 = 0xbe
                    0x00be                  _IPC13 = 0xbe
                    0x00be                  _IPC13bits = 0xbe
                    0x00c2                  IPC15 = 0xc2
                    0x00c2                  _IPC15 = 0xc2
                    0x00c2                  _IPC15bits = 0xc2
                    0x00c4                  IPC16 = 0xc4
                    0x00c4                  _IPC16 = 0xc4
                    0x00c4                  _IPC16bits = 0xc4
                    0x0100                  TMR1 = 0x100
                    0x0100                  _TMR1 = 0x100
                    0x0102                  PR1 = 0x102
                    0x0102                  _PR1 = 0x102
                    0x0104                  T1CON = 0x104
                    0x0104                  _T1CON = 0x104
                    0x0104                  _T1CONbits = 0x104
                    0x0106                  TMR2 = 0x106
                    0x0106                  _TMR2 = 0x106
                    0x0108                  TMR3HLD = 0x108
                    0x0108                  _TMR3HLD = 0x108
                    0x010a                  TMR3 = 0x10a
                    0x010a                  _TMR3 = 0x10a
                    0x010c                  PR2 = 0x10c
                    0x010c                  _PR2 = 0x10c
                    0x010e                  PR3 = 0x10e
                    0x010e                  _PR3 = 0x10e
                    0x0110                  T2CON = 0x110
                    0x0110                  _T2CON = 0x110
                    0x0110                  _T2CONbits = 0x110
                    0x0112                  T3CON = 0x112
                    0x0112                  _T3CON = 0x112
                    0x0112                  _T3CONbits = 0x112
                    0x0114                  TMR4 = 0x114
                    0x0114                  _TMR4 = 0x114
                    0x0116                  TMR5HLD = 0x116
                    0x0116                  _TMR5HLD = 0x116
                    0x0118                  TMR5 = 0x118
                    0x0118                  _TMR5 = 0x118
                    0x011a                  PR4 = 0x11a
                    0x011a                  _PR4 = 0x11a
                    0x011c                  PR5 = 0x11c
                    0x011c                  _PR5 = 0x11c
                    0x011e                  T4CON = 0x11e
                    0x011e                  _T4CON = 0x11e
                    0x011e                  _T4CONbits = 0x11e
                    0x0120                  T5CON = 0x120
                    0x0120                  _T5CON = 0x120
                    0x0120                  _T5CONbits = 0x120
                    0x0140                  IC1BUF = 0x140
                    0x0140                  _IC1BUF = 0x140
                    0x0142                  IC1CON = 0x142
                    0x0142                  _IC1CON = 0x142
                    0x0142                  _IC1CONbits = 0x142
                    0x0144                  IC2BUF = 0x144
                    0x0144                  _IC2BUF = 0x144
                    0x0146                  IC2CON = 0x146
                    0x0146                  _IC2CON = 0x146
                    0x0146                  _IC2CONbits = 0x146
                    0x0148                  IC3BUF = 0x148
                    0x0148                  _IC3BUF = 0x148
                    0x014a                  IC3CON = 0x14a
                    0x014a                  _IC3CON = 0x14a
                    0x014a                  _IC3CONbits = 0x14a
                    0x014c                  IC4BUF = 0x14c
                    0x014c                  _IC4BUF = 0x14c
                    0x014e                  IC4CON = 0x14e
                    0x014e                  _IC4CON = 0x14e
                    0x014e                  _IC4CONbits = 0x14e
                    0x0150                  IC5BUF = 0x150
                    0x0150                  _IC5BUF = 0x150
                    0x0152                  IC5CON = 0x152
                    0x0152                  _IC5CON = 0x152
                    0x0152                  _IC5CONbits = 0x152
                    0x0180                  OC1RS = 0x180
                    0x0180                  _OC1RS = 0x180
                    0x0182                  OC1R = 0x182
                    0x0182                  _OC1R = 0x182
                    0x0184                  OC1CON = 0x184
                    0x0184                  _OC1CON = 0x184
                    0x0184                  _OC1CONbits = 0x184
                    0x0186                  OC2RS = 0x186
                    0x0186                  _OC2RS = 0x186
                    0x0188                  OC2R = 0x188
                    0x0188                  _OC2R = 0x188
                    0x018a                  OC2CON = 0x18a
                    0x018a                  _OC2CON = 0x18a
                    0x018a                  _OC2CONbits = 0x18a
                    0x018c                  OC3RS = 0x18c
                    0x018c                  _OC3RS = 0x18c
                    0x018e                  OC3R = 0x18e
                    0x018e                  _OC3R = 0x18e
                    0x0190                  OC3CON = 0x190
                    0x0190                  _OC3CON = 0x190
                    0x0190                  _OC3CONbits = 0x190
                    0x0192                  OC4RS = 0x192
                    0x0192                  _OC4RS = 0x192
                    0x0194                  OC4R = 0x194
                    0x0194                  _OC4R = 0x194
                    0x0196                  OC4CON = 0x196
                    0x0196                  _OC4CON = 0x196
                    0x0196                  _OC4CONbits = 0x196
                    0x0198                  OC5RS = 0x198
                    0x0198                  _OC5RS = 0x198
                    0x019a                  OC5R = 0x19a
                    0x019a                  _OC5R = 0x19a
                    0x019c                  OC5CON = 0x19c
                    0x019c                  _OC5CON = 0x19c
                    0x019c                  _OC5CONbits = 0x19c
                    0x0200                  I2C1RCV = 0x200
                    0x0200                  _I2C1RCV = 0x200
                    0x0202                  I2C1TRN = 0x202
                    0x0202                  _I2C1TRN = 0x202
                    0x0204                  I2C1BRG = 0x204
                    0x0204                  _I2C1BRG = 0x204
                    0x0206                  I2C1CON = 0x206
                    0x0206                  _I2C1CON = 0x206
                    0x0206                  _I2C1CONbits = 0x206
                    0x0208                  I2C1STAT = 0x208
                    0x0208                  _I2C1STAT = 0x208
                    0x0208                  _I2C1STATbits = 0x208
                    0x020a                  I2C1ADD = 0x20a
                    0x020a                  _I2C1ADD = 0x20a
                    0x020c                  I2C1MSK = 0x20c
                    0x020c                  _I2C1MSK = 0x20c
                    0x0210                  I2C2RCV = 0x210
                    0x0210                  _I2C2RCV = 0x210
                    0x0212                  I2C2TRN = 0x212
                    0x0212                  _I2C2TRN = 0x212
                    0x0214                  I2C2BRG = 0x214
                    0x0214                  _I2C2BRG = 0x214
                    0x0216                  I2C2CON = 0x216
                    0x0216                  _I2C2CON = 0x216
                    0x0216                  _I2C2CONbits = 0x216
                    0x0218                  I2C2STAT = 0x218
                    0x0218                  _I2C2STAT = 0x218
                    0x0218                  _I2C2STATbits = 0x218
                    0x021a                  I2C2ADD = 0x21a
                    0x021a                  _I2C2ADD = 0x21a
                    0x021c                  I2C2MSK = 0x21c
                    0x021c                  _I2C2MSK = 0x21c
                    0x0220                  U1MODE = 0x220
                    0x0220                  _U1MODE = 0x220
                    0x0220                  _U1MODEbits = 0x220
                    0x0222                  U1STA = 0x222
                    0x0222                  _U1STA = 0x222
                    0x0222                  _U1STAbits = 0x222
                    0x0224                  U1TXREG = 0x224
                    0x0224                  _U1TXREG = 0x224
                    0x0226                  U1RXREG = 0x226
                    0x0226                  _U1RXREG = 0x226
                    0x0228                  U1BRG = 0x228
                    0x0228                  _U1BRG = 0x228
                    0x0230                  U2MODE = 0x230
                    0x0230                  _U2MODE = 0x230
                    0x0230                  _U2MODEbits = 0x230
                    0x0232                  U2STA = 0x232
                    0x0232                  _U2STA = 0x232
                    0x0232                  _U2STAbits = 0x232
                    0x0234                  U2TXREG = 0x234
                    0x0234                  _U2TXREG = 0x234
                    0x0236                  U2RXREG = 0x236
                    0x0236                  _U2RXREG = 0x236
                    0x0238                  U2BRG = 0x238
                    0x0238                  _U2BRG = 0x238
                    0x0240                  SPI1STAT = 0x240
                    0x0240                  _SPI1STAT = 0x240
                    0x0240                  _SPI1STATbits = 0x240
                    0x0242                  SPI1CON1 = 0x242
                    0x0242                  _SPI1CON1 = 0x242
                    0x0242                  _SPI1CON1bits = 0x242
                    0x0244                  SPI1CON2 = 0x244
                    0x0244                  _SPI1CON2 = 0x244
                    0x0244                  _SPI1CON2bits = 0x244
                    0x0248                  SPI1BUF = 0x248
                    0x0248                  _SPI1BUF = 0x248
                    0x0260                  SPI2STAT = 0x260
                    0x0260                  _SPI2STAT = 0x260
                    0x0260                  _SPI2STATbits = 0x260
                    0x0262                  SPI2CON1 = 0x262
                    0x0262                  _SPI2CON1 = 0x262
                    0x0262                  _SPI2CON1bits = 0x262
                    0x0264                  SPI2CON2 = 0x264
                    0x0264                  _SPI2CON2 = 0x264
                    0x0264                  _SPI2CON2bits = 0x264
                    0x0268                  SPI2BUF = 0x268
                    0x0268                  _SPI2BUF = 0x268
                    0x02c6                  TRISB = 0x2c6
                    0x02c6                  _TRISB = 0x2c6
                    0x02c6                  _TRISBbits = 0x2c6
                    0x02c8                  PORTB = 0x2c8
                    0x02c8                  _PORTB = 0x2c8
                    0x02c8                  _PORTBbits = 0x2c8
                    0x02ca                  LATB = 0x2ca
                    0x02ca                  _LATB = 0x2ca
                    0x02ca                  _LATBbits = 0x2ca
                    0x02cc                  TRISC = 0x2cc
                    0x02cc                  _TRISC = 0x2cc
                    0x02cc                  _TRISCbits = 0x2cc
                    0x02ce                  PORTC = 0x2ce
                    0x02ce                  _PORTC = 0x2ce
                    0x02ce                  _PORTCbits = 0x2ce
                    0x02d0                  LATC = 0x2d0
                    0x02d0                  _LATC = 0x2d0
                    0x02d0                  _LATCbits = 0x2d0
                    0x02d2                  TRISD = 0x2d2
                    0x02d2                  _TRISD = 0x2d2
                    0x02d2                  _TRISDbits = 0x2d2
                    0x02d4                  PORTD = 0x2d4
                    0x02d4                  _PORTD = 0x2d4
                    0x02d4                  _PORTDbits = 0x2d4
                    0x02d6                  LATD = 0x2d6
                    0x02d6                  _LATD = 0x2d6
                    0x02d6                  _LATDbits = 0x2d6
                    0x02d8                  TRISE = 0x2d8
                    0x02d8                  _TRISE = 0x2d8
                    0x02d8                  _TRISEbits = 0x2d8
                    0x02da                  PORTE = 0x2da
                    0x02da                  _PORTE = 0x2da
                    0x02da                  _PORTEbits = 0x2da
                    0x02dc                  LATE = 0x2dc
                    0x02dc                  _LATE = 0x2dc
                    0x02dc                  _LATEbits = 0x2dc
                    0x02de                  TRISF = 0x2de
                    0x02de                  _TRISF = 0x2de
                    0x02de                  _TRISFbits = 0x2de
                    0x02e0                  PORTF = 0x2e0
                    0x02e0                  _PORTF = 0x2e0
                    0x02e0                  _PORTFbits = 0x2e0
                    0x02e2                  LATF = 0x2e2
                    0x02e2                  _LATF = 0x2e2
                    0x02e2                  _LATFbits = 0x2e2
                    0x02e4                  TRISG = 0x2e4
                    0x02e4                  _TRISG = 0x2e4
                    0x02e4                  _TRISGbits = 0x2e4
                    0x02e6                  PORTG = 0x2e6
                    0x02e6                  _PORTG = 0x2e6
                    0x02e6                  _PORTGbits = 0x2e6
                    0x02e8                  LATG = 0x2e8
                    0x02e8                  _LATG = 0x2e8
                    0x02e8                  _LATGbits = 0x2e8
                    0x02fc                  PADCFG1 = 0x2fc
                    0x02fc                  _PADCFG1 = 0x2fc
                    0x02fc                  _PADCFG1bits = 0x2fc
                    0x0300                  ADC1BUF0 = 0x300
                    0x0300                  _ADC1BUF0 = 0x300
                    0x0302                  ADC1BUF1 = 0x302
                    0x0302                  _ADC1BUF1 = 0x302
                    0x0304                  ADC1BUF2 = 0x304
                    0x0304                  _ADC1BUF2 = 0x304
                    0x0306                  ADC1BUF3 = 0x306
                    0x0306                  _ADC1BUF3 = 0x306
                    0x0308                  ADC1BUF4 = 0x308
                    0x0308                  _ADC1BUF4 = 0x308
                    0x030a                  ADC1BUF5 = 0x30a
                    0x030a                  _ADC1BUF5 = 0x30a
                    0x030c                  ADC1BUF6 = 0x30c
                    0x030c                  _ADC1BUF6 = 0x30c
                    0x030e                  ADC1BUF7 = 0x30e
                    0x030e                  _ADC1BUF7 = 0x30e
                    0x0310                  ADC1BUF8 = 0x310
                    0x0310                  _ADC1BUF8 = 0x310
                    0x0312                  ADC1BUF9 = 0x312
                    0x0312                  _ADC1BUF9 = 0x312
                    0x0314                  ADC1BUFA = 0x314
                    0x0314                  _ADC1BUFA = 0x314
                    0x0316                  ADC1BUFB = 0x316
                    0x0316                  _ADC1BUFB = 0x316
                    0x0318                  ADC1BUFC = 0x318
                    0x0318                  _ADC1BUFC = 0x318
                    0x031a                  ADC1BUFD = 0x31a
                    0x031a                  _ADC1BUFD = 0x31a
                    0x031c                  ADC1BUFE = 0x31c
                    0x031c                  _ADC1BUFE = 0x31c
                    0x031e                  ADC1BUFF = 0x31e
                    0x031e                  _ADC1BUFF = 0x31e
                    0x0320                  AD1CON1 = 0x320
                    0x0320                  _AD1CON1 = 0x320
                    0x0320                  _AD1CON1bits = 0x320
                    0x0322                  AD1CON2 = 0x322
                    0x0322                  _AD1CON2 = 0x322
                    0x0322                  _AD1CON2bits = 0x322
                    0x0324                  AD1CON3 = 0x324
                    0x0324                  _AD1CON3 = 0x324
                    0x0324                  _AD1CON3bits = 0x324
                    0x0328                  AD1CHS = 0x328
                    0x0328                  _AD1CHS = 0x328
                    0x0328                  _AD1CHSbits = 0x328
                    0x032c                  AD1PCFG = 0x32c
                    0x032c                  _AD1PCFG = 0x32c
                    0x032c                  _AD1PCFGbits = 0x32c
                    0x0330                  AD1CSSL = 0x330
                    0x0330                  _AD1CSSL = 0x330
                    0x0330                  _AD1CSSLbits = 0x330
                    0x0600                  PMCON = 0x600
                    0x0600                  _PMCON = 0x600
                    0x0600                  _PMCONbits = 0x600
                    0x0602                  PMMODE = 0x602
                    0x0602                  _PMMODE = 0x602
                    0x0602                  _PMMODEbits = 0x602
                    0x0604                  PMADDR = 0x604
                    0x0604                  _PMADDR = 0x604
                    0x0604                  _PMADDRbits = 0x604
                    0x0604                  PMDOUT1 = 0x604
                    0x0604                  _PMDOUT1 = 0x604
                    0x0606                  PMDOUT2 = 0x606
                    0x0606                  _PMDOUT2 = 0x606
                    0x0608                  PMDIN1 = 0x608
                    0x0608                  _PMDIN1 = 0x608
                    0x060a                  PMDIN2 = 0x60a
                    0x060a                  _PMDIN2 = 0x60a
                    0x060c                  PMAEN = 0x60c
                    0x060c                  _PMAEN = 0x60c
                    0x060c                  _PMAENbits = 0x60c
                    0x060e                  PMSTAT = 0x60e
                    0x060e                  _PMSTAT = 0x60e
                    0x060e                  _PMSTATbits = 0x60e
                    0x0620                  ALRMVAL = 0x620
                    0x0620                  _ALRMVAL = 0x620
                    0x0622                  ALCFGRPT = 0x622
                    0x0622                  _ALCFGRPT = 0x622
                    0x0622                  _ALCFGRPTbits = 0x622
                    0x0624                  RTCVAL = 0x624
                    0x0624                  _RTCVAL = 0x624
                    0x0626                  RCFGCAL = 0x626
                    0x0626                  _RCFGCAL = 0x626
                    0x0626                  _RCFGCALbits = 0x626
                    0x0630                  CMCON = 0x630
                    0x0630                  _CMCON = 0x630
                    0x0630                  _CMCONbits = 0x630
                    0x0632                  CVRCON = 0x632
                    0x0632                  _CVRCON = 0x632
                    0x0632                  _CVRCONbits = 0x632
                    0x0640                  CRCCON = 0x640
                    0x0640                  _CRCCON = 0x640
                    0x0640                  _CRCCONbits = 0x640
                    0x0642                  CRCXOR = 0x642
                    0x0642                  _CRCXOR = 0x642
                    0x0644                  CRCDAT = 0x644
                    0x0644                  _CRCDAT = 0x644
                    0x0646                  CRCWDAT = 0x646
                    0x0646                  _CRCWDAT = 0x646
                    0x06c6                  ODCB = 0x6c6
                    0x06c6                  _ODCB = 0x6c6
                    0x06c6                  _ODCBbits = 0x6c6
                    0x06cc                  ODCC = 0x6cc
                    0x06cc                  _ODCC = 0x6cc
                    0x06cc                  _ODCCbits = 0x6cc
                    0x06d2                  ODCD = 0x6d2
                    0x06d2                  _ODCD = 0x6d2
                    0x06d2                  _ODCDbits = 0x6d2
                    0x06d8                  ODCE = 0x6d8
                    0x06d8                  _ODCE = 0x6d8
                    0x06d8                  _ODCEbits = 0x6d8
                    0x06de                  ODCF = 0x6de
                    0x06de                  _ODCF = 0x6de
                    0x06de                  _ODCFbits = 0x6de
                    0x06e4                  ODCG = 0x6e4
                    0x06e4                  _ODCG = 0x6e4
                    0x06e4                  _ODCGbits = 0x6e4
                    0x0740                  RCON = 0x740
                    0x0740                  _RCON = 0x740
                    0x0740                  _RCONbits = 0x740
                    0x0742                  OSCCON = 0x742
                    0x0742                  _OSCCON = 0x742
                    0x0742                  _OSCCONbits = 0x742
                    0x0744                  CLKDIV = 0x744
                    0x0744                  _CLKDIV = 0x744
                    0x0744                  _CLKDIVbits = 0x744
                    0x0748                  OSCTUN = 0x748
                    0x0748                  _OSCTUN = 0x748
                    0x0748                  _OSCTUNbits = 0x748
                    0x0760                  NVMCON = 0x760
                    0x0760                  _NVMCON = 0x760
                    0x0760                  _NVMCONbits = 0x760
                    0x0766                  NVMKEY = 0x766
                    0x0766                  _NVMKEY = 0x766
                    0x0770                  PMD1 = 0x770
                    0x0770                  _PMD1 = 0x770
                    0x0770                  _PMD1bits = 0x770
                    0x0772                  PMD2 = 0x772
                    0x0772                  _PMD2 = 0x772
                    0x0772                  _PMD2bits = 0x772
                    0x0774                  PMD3 = 0x774
                    0x0774                  _PMD3 = 0x774
                    0x0774                  _PMD3bits = 0x774
                    0x0140                  IC1 = 0x140
                    0x0140                  _IC1 = 0x140
                    0x0144                  IC2 = 0x144
                    0x0144                  _IC2 = 0x144
                    0x0148                  IC3 = 0x148
                    0x0148                  _IC3 = 0x148
                    0x014c                  IC4 = 0x14c
                    0x014c                  _IC4 = 0x14c
                    0x0150                  IC5 = 0x150
                    0x0150                  _IC5 = 0x150
                    0x0180                  OC1 = 0x180
                    0x0180                  _OC1 = 0x180
                    0x0186                  OC2 = 0x186
                    0x0186                  _OC2 = 0x186
                    0x018c                  OC3 = 0x18c
                    0x018c                  _OC3 = 0x18c
                    0x0192                  OC4 = 0x192
                    0x0192                  _OC4 = 0x192
                    0x0198                  OC5 = 0x198
                    0x0198                  _OC5 = 0x198
                    0x0240                  SPI1 = 0x240
                    0x0240                  _SPI1 = 0x240
                    0x0260                  SPI2 = 0x260
                    0x0260                  _SPI2 = 0x260
                    0x0220                  UART1 = 0x220
                    0x0220                  _UART1 = 0x220
                    0x0230                  UART2 = 0x230
                    0x0230                  _UART2 = 0x230
START GROUP
LOAD c:/program files/microchip/mplab c30/bin/../lib\libpic30-coff.a
LOAD c:/program files/microchip/mplab c30/bin/../lib\libm-coff.a
LOAD c:/program files/microchip/mplab c30/bin/../lib\libc-coff.a
END GROUP
OUTPUT(EVBs.cof coff-pic30)
LOAD jump_table
LOAD data_init
LOAD default_isr

.const            0x008736       0x4886
 .const           0x008736       0x18c0 loopback.o
 .const           0x009ff6        0x486 ping_app.o
 .const           0x00a47c        0x6fc webserver.o
 .const           0x00ab78        0x15a config.o
 .const           0x00acd2        0x1ca evb.o
 .const           0x00ae9c        0x4b8 manage.o
 .const           0x00b354         0x48 SEEP.o
 .const           0x00b39c        0xdb6 dhcp.o
 .const           0x00c152        0x820 dns.o
 .const           0x00c972        0x234 httpd.o
 .const           0x00cba6        0x270 ping.o
 .const           0x00ce16         0xd0 main.o
 .const           0x00cee6          0x4 serial.o
 .const           0x00ceea         0x52 romfs.o
 .const           0x00cf3c         0x22 sockutil.o
 .const           0x00cf5e         0x5e w5100.o

.ndata              0x0800       0x1000
 .ndata             0x0800       0x1000 webserver.o
                    0x0800                  data_buf1
                    0x1000                  data_buf2

.ndata              0x1800         0x88
 .ndata             0x1800         0x88 c:/program files/microchip/mplab c30/bin/../lib\libc-coff.a(xfiles.o)
                    0x1800                  _Files
                    0x1810                  _Stderr
                    0x1838                  _Stdout
                    0x1860                  _Stdin

.nbss               0x1888         0x46
 .nbss              0x1888         0x46 config.o
                    0x1888                  SysInfo
                    0x1892                  NetConf
                    0x18ac                  ChConf

.ndata              0x18ce         0x40
 .ndata             0x18ce         0x40 md5.o

.ndata              0x190e         0x3a
 .ndata             0x190e         0x3a romfs.o
                    0x1946                  romfl_list

.nbss               0x1948         0x34
 .nbss              0x1948         0x34 w5100.o

.ndata              0x197c         0x32
 .ndata             0x197c         0x32 dhcp.o
                    0x197c                  GET_DNS_IP
                    0x1980                  HOST_NAME
                    0x199e                  GET_SIP
                    0x19a2                  DHCP_SIP
                    0x19a6                  DHCP_REAL_SIP
                    0x19aa                  dhcp_ip_update
                    0x19ac                  dhcp_ip_conflict

.nbss               0x19ae         0x2a
 .nbss              0x19ae         0x2a dhcp.o
                    0x19ae                  SRC_MAC_ADDR
                    0x19b4                  GET_SN_MASK
                    0x19b8                  GET_GW_IP
                    0x19bc                  OLD_SIP
                    0x19c0                  dhcp_state
                    0x19c1                  retry_count
                    0x19c2                  DHCP_timeout
                    0x19c4                  lease_time
                    0x19c8                  dhcp_time
                    0x19cc                  next_dhcp_time
                    0x19d0                  DHCP_XID
                    0x19d4                  DHCPC_SOCK
                    0x19d6                  pRIPMSG

.nbss               0x19d8         0x28
 .nbss              0x19d8         0x28 serial.o
                    0x19d8                  sio_rxd
                    0x19f8                  sio_head
                    0x19fa                  sio_tail
                    0x19fc                  uart_handler

.nbss               0x1a00         0x22
 .nbss              0x1a00         0x22 evb.o
                    0x1a00                  evb_lcd_text

.ndata              0x1a22         0x22
 .ndata             0x1a22         0x22 c:/program files/microchip/mplab c30/bin/../lib\libc-coff.a(xlitob.o)

.nbss               0x1a44         0x20
 .nbss              0x1a44         0x20 sockutil.o

.ndata              0x1a64         0x12
 .ndata             0x1a64         0x12 c:/program files/microchip/mplab c30/bin/../lib\libc-coff.a(xprintf.io)

.nbss               0x1a76          0xa
 .nbss              0x1a76          0xa dns.o
                    0x1a76                  dns_buf
                    0x1a78                  get_domain_name
                    0x1a7a                  get_domain_ip
                    0x1a7e                  query_data

.nbss               0x1a80          0x8
 .nbss              0x1a80          0x8 channel.o
                    0x1a80                  ChannelHandler

.ndata              0x1a88          0x6
 .ndata             0x1a88          0x6 channel.o
                    0x1a88                  sock_flag
                    0x1a89                  bchannel_start

.nbss               0x1a8e          0x6
 .nbss              0x1a8e          0x6 timer.o
                    0x1a8e                  sys_tick_5ms
                    0x1a90                  sys_tick_1s
                    0x1a92                  TIMER_IRQS

.ndata              0x1a94          0x6
 .ndata             0x1a94          0x6 c:/program files/microchip/mplab c30/bin/../lib\libc-coff.a(malloc.o)
                    0x1a94                  _Size_block
                    0x1a96                  _Aldata

.nbss               0x1a9a          0x4
 .nbss              0x1a9a          0x4 webserver.o
                    0x1a9a                  http_response
                    0x1a9c                  http_request

.ndata              0x1a9e          0x4
 .ndata             0x1a9e          0x4 ping.o

.nbss               0x1aa2          0x2
 .nbss              0x1aa2          0x2 socket.o

.ndata              0x1aa4          0x2
 .ndata             0x1aa4          0x2 dns.o
                    0x1aa4                  dns_id

.ndata              0x1aa6          0x2
 .ndata             0x1aa6          0x2 c:/program files/microchip/mplab c30/bin/../lib\libc-coff.a(strtok.o)

.nbss               0x1aa8          0x2
 .nbss              0x1aa8          0x2 c:/program files/microchip/mplab c30/bin/../lib\libc-coff.a(strtok.o)

.nbss               0x1aaa          0x2
 .nbss              0x1aaa          0x2 c:/program files/microchip/mplab c30/bin/../lib\libc-coff.a(fclose.o)

.nbss               0x1aac          0x2
 .nbss              0x1aac          0x2 c:/program files/microchip/mplab c30/bin/../lib\libpic30-coff.a(brk.o)
                    0x1aac                  __curbrk

.dconst             0x1aae          0x8
 .dconst            0x1aae          0x8 c:/program files/microchip/mplab c30/bin/../lib\libc-coff.a(xprintf.io)

.dconst             0x1ab6          0x2
 .dconst            0x1ab6          0x2 c:/program files/microchip/mplab c30/bin/../lib\libc-coff.a(strtok.o)

.prog             0x00cfbc       0x281e
 .prog            0x00cfbc       0x281e romfs.o
                  0x00cfbc                  file0data
                  0x00d8d4                  file1data
                  0x00dfbe                  file2data
                  0x00ee10                  file3data
                  0x00f3bc                  file4data
                  0x00f490                  file5data
                  0x00f574                  file6data

.dinit            0x00f7da        0xc64
 .dinit           0x00f7da        0xc64 data_init

.isr              0x01043e          0x2
 .isr             0x01043e          0x2 default_isr
                  0x01043e                  _DefaultInterrupt
